:020000040800F2
:100000002837002001010008252A0008EF1E0008FB
:10001000212A0008DD050008A536000800000000C0
:10002000000000000000000000000000A12E0008F9
:100030002D06000800000000B72B0008F92E00086C
:100040001B0100081B0100081B010008492E0008C5
:100050001B0100081B0100081B0100081B01000810
:100060001B0100081B0100081B0100081B01000800
:100070001B0100081B0100081B0100081B010008F0
:10008000E1050008F10500081B0100081B0100083C
:100090001B0100081B0100081B0100081B010008D0
:1000A0001B0100081B0100081B0100081B010008C0
:1000B0005D2F0008E12F0008453000081B010008F3
:1000C0001B0100081B0100081B0100081B010008A0
:1000D0001B0100081B010008FD350008113600084F
:1000E0001B0100081B0100081B010008DFF80CD0F1
:1000F00000F034F900480047B963000828370020B1
:100100000648804706480047FEE7FEE7FEE7FEE7B1
:10011000FEE7FEE7FEE7FEE7FEE7FEE7052F000845
:10012000ED000008202A04DB203A21FA02F0002129
:10013000704721FA02F3D040C2F1200291400843F7
:100140001946704710B540EA01040346A40703D0DE
:1001500009E010C9121F10C3042AFAD203E011F8F3
:10016000014B03F8014B521EF9D210BDD2B201E08F
:1001700000F8012B491EFBD270470022F6E710B5AC
:1001800013460A4604461946FFF7F0FF204610BD05
:1001900030B505462A460B4612F8010B13F8014B01
:1001A00008B1A042F8D01CB1002802D06D1CF1E7C4
:1001B000284630BD10B5044604E00B7800F8013B3A
:1001C00003B1491C521EF8D2204610BDCAB2401ECF
:1001D00010F8011F8A4202D00029F9D1002070478F
:1001E000421C10F8011B0029FBD1801A704710B582
:1001F000002200E0521C835C8C5CA34201D1002BE6
:10020000F8D1D8B2E1B2401A10BD30B50446002092
:10021000034600E05B1C934203D2E05CCD5C401BD4
:10022000F8D030BD034611F8012B00F8012B002A4D
:10023000F9D11846704730B505460020034600E066
:100240005B1C934205D2EC5CC85C201A01D1002CE7
:10025000F6D130BD70B5064603F0D4FA0468054601
:100260000A220021304600F040F82C6070BD70B5C5
:10027000064603F0C7FA046805460A220021304604
:1002800000F033F82C6070BD2DE9F05F05460020CA
:1002900092469B4688460646814640241BE02846F7
:1002A000414647462246FFF73DFF53465A46C01A8D
:1002B000914110D311461846224600F061F82D1ADC
:1002C00067EB01084F4622460120002100F058F854
:1002D00017EB00094E41201EA4F10104DFDC484663
:1002E00031462A464346BDE8F09F2DE9F047914646
:1002F0000F4680460446002614F8015B2DB100F03D
:100300004FF80068405DC007F6D12B2D02D02D2D8F
:1003100018D0641E4A463946204600F045F827B1F9
:100320003968A14201D1C7F8008071054FF002047D
:100330000BD54042002803DD03F064FA0460A007F7
:10034000BDE8F08746F48066E4E70028F8DA03F0B9
:1003500059FA04606FF00040F2E70000064C074DC8
:1003600006E0E06840F0010394E807009847103485
:10037000AC42F6D3FFF7BEFEF8A5000818A60008A9
:10038000202A04DB203A00FA02F100207047914055
:10039000C2F1200320FA03F3194390407047000094
:1003A0000048704754A200082DE9F05F82460078AB
:1003B000002715468B460AF10104B946302801D0C2
:1003C0009DB113E014F8010B0127782803D05828B9
:1003D00001D045B10AE00DB1102D07D1002710253D
:1003E00014F8010B02E0082500E00A250026B046BB
:1003F0000EE005FB080005FB06F1012701EB1046A6
:100400001FFA80F8B6F5803F00D3B94614F8010B07
:10041000294600F018F80028EBDABBF1000F05D0F0
:100420000FB1641E00E05446CBF80040B9F1000F54
:1004300006D003F0E7F902210160C81EBDE8F09F75
:1004400048EA0640FAE73A2800D2303820F0200285
:10045000412A01D3A2F13700884201D34FF0FF3087
:10046000704770B58C1810F8015B15F0070301D1C7
:1004700010F8013B2A1106D110F8012B03E010F807
:10048000016B01F8016B5B1EF9D12B0705D400232A
:10049000521E0DD401F8013BFAE710F8013BCB1ACC
:1004A000921C03E013F8015B01F8015B521EF9D5C1
:1004B000A142D8D3002070BD10B5FF2000F028F86D
:1004C0000446552C01D1002010BD5521FF2000F01D
:1004D0005DF8FF2000F01CF80446552C01D10020E7
:1004E000F2E70120F0E710B501F02CFD10BD70B56A
:1004F00006460C46154608E03046721C96B200F0DF
:1005000007F804F8010B681E85B2002DF4D170BD08
:1005100070B50446002601F0F5FD2546E11704EB11
:1005200011610912A02202EB4101C8B201F0B6FD2F
:1005300001F034FEE11704EB11610912A4EB012173
:10054000C8B201F0ABFD01F029FE01F0DBFDA120F6
:1005500001F0A4FD01F022FE002001F067FD064637
:1005600001F0F6FD304670BD70B505460C461646E6
:1005700006E02178284600F009F8681C85B2641C62
:10058000301EA6F101018EB2F3D170BD70B50446E4
:100590000E4601F0B7FD2546E11704EB1161091283
:1005A000A02202EB4101C8B201F078FD01F0F6FD96
:1005B000E11704EB11610912A4EB0121C8B201F0AB
:1005C0006DFD01F0EBFD304601F068FD01F0E6FD48
:1005D00001F0BEFD0A2004F031FA70BD00BFFEE755
:1005E00010B5024800F030F910BD000040050020B1
:1005F00010B5024800F028F910BD0000FC040020EE
:1006000030B590F840500124AC40C56B6C60046874
:1006100063604468102C04D10468A2600468E1603F
:1006200003E00468A1600468E26030BD704770B503
:1006300004460D461646204600F061F810B14FF012
:10064000FF3070BDD4F8CC0500EB400004EB001186
:100650002846FFF7E7FDD4F8CC0500EB400204F58F
:10066000F07000EB42113046FFF7DCFDD4F8CC050A
:10067000401C0A21B0FBF1F201FB1200C4F8CC05CA
:10068000D4F8D005401EC4F8D0050120D9E70021D8
:10069000C0F8C815C0F8CC15C0F8D015704770B5B3
:1006A00004460E461546204600F032F810B14FF0D1
:1006B000FF3070BDD4F8C81501EB410104EB011007
:1006C0003146FFF7AFFDD4F8C81501EB410204F540
:1006D000F07101EB42102946FFF7A4FDD4F8C805DC
:1006E000401C0A21B0FBF1F201FB1200C4F8C8055E
:1006F000D4F8D005401CC4F8D0050120D9E7014644
:10070000D1F8D00508B9012070470020FCE70000AF
:1007100010B50446012003F043F8962004F09AF93E
:100720000A2209A0D4F8D01503F048F8962004F066
:1007300091F9002003F034F8D4F8D0050A2801D14B
:10074000012010BD0020FCE76669666F20757365A7
:10075000643A25642F25640A000000000146002049
:100760000A68126822F00E020B681A600A681268A2
:1007700022F001020B681A6091F8403001229A4081
:10078000CB6B5A60012281F8212000BF002281F842
:10079000202000BF7047000070B50446002594F883
:1007A0002100022803D00420A063012548E020682E
:1007B000006820F00E00216808602068006820F0C2
:1007C0000100216808601F492068884201D101208A
:1007D00026E01C4914312068884201D110201FE016
:1007E000184928312068884201D1801518E0154940
:1007F0003C312068884201D1801411E01149503108
:100800002068884202D14FF4803009E00D496431FC
:100810002068884202D14FF4801001E04FF08070D0
:10082000084908394860012084F8210000BF0020F1
:1008300084F8200000BF606B10B12046616B8847D0
:10084000284670BD0800024070B50446E06B05689C
:100850002068066894F8401004208840284000284A
:1008600046D006F00400002842D02068006800F05E
:10087000200028B92068006820F004002168086082
:1008800057492068884201D1042027E05449143197
:100890002068884201D1402020E051492831206859
:1008A000884201D1001519E04D493C312068884249
:1008B00002D14FF4804011E049495031206888420C
:1008C00002D14FF4802009E0454964312068884214
:1008D00002D14FF4800001E04FF0806040490839B8
:1008E0004860E06A00287AD02046E16A884776E0CE
:1008F00094F84010022088402840A0B306F002007F
:1009000088B32068006800F0200040B920680068C3
:1009100020F00A0021680860012084F82100304995
:100920002068884201D1022028E02D491431206836
:10093000884201D1202021E02949283120688842BD
:1009400001D140151AE026493C312068884202D185
:100950004FF4005012E0224950312068884203D100
:100960004FF400300AE017E01D49643120688842E6
:1009700002D14FF4001001E04FF00070184908391F
:10098000486000BF002084F8200000BFA06A30B398
:100990002046A16A884722E094F840100820884049
:1009A0002840E0B106F00800C8B12068006820F0D7
:1009B0000E002168086094F8401001208840E16B27
:1009C00048600120A06384F8210000BF002084F863
:1009D000200000BF206B10B12046216B884770BDFE
:1009E000080002400146002209B901207047184B57
:1009F0000868C01A1423B0FBF3F0800008641448A0
:100A00000838C863022081F821000868026843F6AC
:100A1000F0708243D1E901031843CB6818430B6996
:100A200018434B6918438B691843CB691843024339
:100A30000868026000208862C862086348638863AF
:100A4000012081F82100002081F8200000BFCDE7BF
:100A5000080002402DE9F04104460D4616461F46A7
:100A60004FF0000800BF94F82000012802D10220B6
:100A7000BDE8F081012084F8200000BF94F8210037
:100A800001282CD1022084F821000020A0632068D6
:100A9000006820F00100216808603B463246294684
:100AA0002046FFF7ADFDE06A30B12068006840F0F5
:100AB0000E00216808600BE02068006820F0040048
:100AC000216808602068006840F00A00216808601A
:100AD0002068006840F001002168086006E000BF5F
:100AE000002084F8200000BF4FF002084046BFE716
:100AF0002DE9F847034600240020002584460027FE
:100B000000226EE14FF0010808FA02F4D1F80080EB
:100B100008EA0400A0427DD1DFF8D0A2D1F8048019
:100B2000A8EB0A09D0453AD014DCB8F1030F50D035
:100B300009DCB8F1000F31D0B8F1010F1CD0B8F1C9
:100B4000020F49D120E0B8F1110F18D0B8F1120FFF
:100B500042D11EE0B9F5881F25D006DCB9F5803FEB
:100B600020D0B9F5801F37D11AE0B9F5001F18D091
:100B7000B9F5041F30D117E0D1F80CC02DE0D1F841
:100B80000C8008F1040C28E0D1F80C8008F1080C66
:100B900023E0D1F80C8008F10C0C1EE000BF00BF70
:100BA00000BF00BF00BF00BFD1F80880B8F1000F40
:100BB00002D14FF0040C0BE0D1F80880B8F1010F1E
:100BC00003D14FF0080C1C6102E04FF0080C5C618F
:100BD00003E04FF0000C00E000BF00BFFF2801D889
:100BE000984601E003F104084646FF2802D84FEA80
:100BF000820803E0A2F108084FEA88084746D6F8C1
:100C000000804FF00F0909FA07F928EA09080CFAE1
:100C100007F900E088E048EA0908C6F80080D1F842
:100C2000048008F08058B8F1805F7DD100BFDFF804
:100C3000C081D8F8188048F00108DFF8B491C9F8ED
:100C40001880C846D8F8188008F00108CDF8008050
:100C500000BF00BF4FEAB9384FEA920958F829504F
:100C60004FEA82784FEA18794FF00F0808FA09F82E
:100C700025EA0805DFF87C81434502D14FF00008E2
:100C800016E0DFF87481434502D14FF001080FE010
:100C9000DFF86881434502D14FF0020808E0DFF831
:100CA0006081434502D14FF0030801E04FF0040892
:100CB0004FEA82794FEA197908FA09F848EA0505F6
:100CC000DFF840814FEA920948F82950D1F80480B2
:100CD00008F48038B8F5803F0AD1DFF82C81D8F8C5
:100CE000008048EA0008DFF82091C9F8008009E098
:100CF000DFF81481D8F8008028EA0008DFF80891AE
:100D0000C9F80080D1F8048008F40038B8F5003F35
:100D100010D1DFF8F48008F10408D8F8008048EA20
:100D20000008DFF8E49000E05AE009F10409C9F88E
:100D300000800DE0DFF8D08008F10408D8F80080CA
:100D400028EA0008DFF8C09009F10409C9F800801A
:100D5000D1F8048008F48018B8F5801F0ED1DFF8B0
:100D6000A88008F10808D8F8008048EA0008DFF8F1
:100D7000989009F10809C9F800800DE0DFF8888033
:100D800008F10808D8F8008028EA0008DFF8789011
:100D900009F10809C9F80080D1F8048008F40018A6
:100DA000B8F5001F0ED1DFF8608008F10C08D8F804
:100DB000008048EA0008DFF8509009F10C09C9F8F2
:100DC00000800DE0DFF8408008F10C08D8F80080C2
:100DD00028EA0008DFF8309009F10C09C9F8008012
:100DE000521C102AFFF48EAEBDE8F88700001110E7
:100DF0000010024000080140000C014000100140BA
:100E00000014014008000140000401400AB10161E2
:100E100001E00B040361704701480068704700005F
:100E2000000000200348006803490978084401498C
:100E300008607047000000200800002010B5084836
:100E4000006840F0100006490860032000F0C2F876
:100E5000002000F007F800F02BF8002010BD000083
:100E60000020024070B504460E4800784FF47A71B5
:100E7000B1FBF0F00C490968B1FBF0F5284600F031
:100E800034FC08B1012070BD102C07D2002221468D
:100E9000501E00F060F80548046001E00120F2E710
:100EA0000020F0E70800002060010020040000207E
:100EB00008B500BF1F48806940F001001D498861E6
:100EC0000846806900F00100009000BF00BF0320C9
:100ED00000F080F8002211466FF00B0000F03BF8A4
:100EE000002211466FF00A0000F035F8002211468A
:100EF0006FF0090000F02FF800221146501F00F09B
:100F00002AF800221146101F00F025F80022114691
:100F1000901E00F020F800221146501E00F01BF831
:100F200000BF0549486820F0E06040F0007048606C
:100F300000BF08BD001002400000014000BF00F0EB
:100F40001F02012191404209920002F1E022C2F801
:100F5000001100BF70472DE9F05F80460D46164630
:100F6000002701F061FD074639462A46334601F065
:100F70000700C0F1070ABAF1040F02D94FF0040AC2
:100F800001E0C0F1070AD14600F1040ABAF1070FE7
:100F900002D24FF0000A01E0A0F1030AD4464FF05C
:100FA000010A0AFA09FAAAF1010A0AEA020A0AFA85
:100FB0000CFA4FF0010B0BFA0CFBABF1010B0BEA37
:100FC000030B4AEA0B042146404601F035FDBDE81B
:100FD000F09F000000BF00F00702064B19684FF6B3
:100FE000FF031940044B0B4343EA0221014B1960F4
:100FF00000BF70470CED00E00000FA0570B5044634
:101000000D4600266248006800F00700A8420ED294
:101010005F48006820F0070028435D4908600846E3
:10102000006800F00700A84201D0012070BD2078C0
:1010300000F00200022807D15648406820F0F00076
:10104000A168084353494860207800F00100002857
:101050005DD06068012806D14E48006800F4003079
:1010600090B90120E2E76068022806D1494800688B
:1010700000F0007040B90120D8E74648006800F051
:10108000020008B90120D1E74248406820F003007F
:10109000616808433F494860FFF7BEFE0646606846
:1010A000012810D108E0FFF7B7FE801B41F288311C
:1010B000884201D90320B9E73648406800F00C00A7
:1010C0000428F0D123E06068022810D108E0FFF77F
:1010D000A3FE801B41F28831884201D90320A5E795
:1010E0002C48406800F00C000828F0D10FE008E020
:1010F000FFF792FE801B41F28831884201D903201C
:1011000094E72448406800F00C000028F0D1204803
:10111000006800F00700A8420ED91D48006820F0C2
:10112000070028431A4908600846006800F00700D5
:10113000A84201D0012079E7207800F004000428BB
:1011400007D11448406820F4E060E1680843114981
:101150004860207800F00800082808D10D48406851
:1011600020F46050216940EAC1000A49486000F05B
:101170003DF808494968C1F30311074A515CC8406A
:10118000064908600020FFF76DFE00204EE70000D2
:10119000002002400010024090A0000860010020E2
:1011A00001480068704700006001002000B5FFF7AB
:1011B000F7FF04494968C1F30221034A515CC84062
:1011C00000BD000000100240A0A0000800B5FFF71D
:1011D000E7FF04494968C1F3C221034A515CC84092
:1011E00000BD000000100240A0A00008F0B585B0CE
:1011F0000FF26C0C9CE8E01001A8A0E8E0101CA520
:101200002D68009500210022002300240020194DA4
:10121000696801F00C05F5B1042D02D0082D19D133
:1012200001E0154819E001ADC1F38346AC5D01F45E
:10123000803555B10F4D6D68C5F340451DF805204B
:101240000D4D6543B5FBF2F302E00C4D04FB05F3D5
:10125000184602E000BF084800BF00BF05B0F0BD5F
:1012600002030405060708090A0B0C0D0E0F1010E7
:10127000010200000010024000127A0000093D0047
:10128000F8B504460025207800F00100002878D049
:10129000F848406800F00C0004280CD0F54840687D
:1012A00000F00C00082811D1F248406800F48030AA
:1012B000B0F5803F0AD1EF48006800F40030002804
:1012C0005FD0606800285CD10120F8BD00BF606875
:1012D000B0F5803F06D1E748006840F48030E5492A
:1012E000086028E0606858B9E248006820F480305F
:1012F000E04908600846006820F4802008601AE091
:101300006068B0F5A02F0BD1DA48006840F4802067
:10131000D84908600846006840F4803008600AE058
:10132000D448006820F48030D2490860084600683C
:1013300020F48020086000BF606888B1FFF76CFD72
:10134000054606E0FFF768FD401B642801D903202D
:10135000BBE7C848006800F400300028F2D010E075
:10136000FFF75AFD054606E0FFF756FD401B6428CF
:1013700001D90320A9E7BF48006800F40030002825
:10138000F2D1207800F00200022857D1B948406815
:1013900000F00C0050B1B748406800F00C0008287D
:1013A00018D1B448406800F4803098B9B14800685A
:1013B00000F0020020B12069012801D0012084E75B
:1013C000AC48006820F0F800616940EAC100A94912
:1013D000086033E02069E8B10120A7490860FFF701
:1013E0001BFD054606E0FFF717FD401B022801D94B
:1013F00003206AE79F48006800F002000028F2D04E
:101400009C48006820F0F800616940EAC1009949F1
:10141000086013E0002098490860FFF7FDFC0546CE
:1014200006E0FFF7F9FC401B022801D903204CE736
:101430009048006800F002000028F2D1207800F007
:10144000080008282DD1A069B8B101208B49086097
:10145000FFF7E2FC054606E0FFF7DEFC401B022832
:1014600001D9032031E78348406A00F002000028D8
:10147000F2D0012001F0D2FB13E000207F49086088
:10148000FFF7CAFC054606E0FFF7C6FC401B022832
:1014900001D9032019E77748406A00F002000028CC
:1014A000F2D1207800F00400042873D1002671489E
:1014B000C06900F0805070B900BF6E48C06940F04C
:1014C00080506C49C8610846C06900F080500090A7
:1014D00000BF00BF01266A48006800F48070B0B900
:1014E0006748006840F4807065490860FFF794FC25
:1014F000054606E0FFF790FC401B642801D9032055
:10150000E3E65F48006800F480700028F2D000BF76
:10151000E068012806D15748006A40F001005549AB
:10152000086227E0E06858B95248006A20F00100DC
:10153000504908620846006A20F00400086219E079
:10154000E06805280BD14B48006A40F00400494987
:1015500008620846006A40F0010008620AE0454857
:10156000006A20F00100434908620846006A20F042
:101570000400086200BFE068A0B1FFF74DFC05461B
:1015800009E0FFF749FC401B41F28831884202D94B
:1015900003209AE622E03748006A00F002000028A3
:1015A000EFD012E0FFF738FC054608E0FFF734FC07
:1015B000401B41F28831884201D9032085E62D483D
:1015C000006A00F002000028F0D1012E05D1294860
:1015D000C06920F080502749C86100BFE069C8B3E6
:1015E0002448406800F00C00082860D0E069022818
:1015F00048D1002020490866FFF70EFC054606E0AA
:10160000FFF70AFC401B022801D903205DE61948B8
:10161000006800F000700028F2D1206AB0F5803F29
:1016200007D11448406820F40030A16808431149EC
:101630004860D4E9080108430E49496821F474114F
:1016400008430C49486001200B490866FFF7E4FB9A
:10165000054607E02DE0FFF7DFFB401B022801D91C
:10166000032032E60348006800F000700028F2D042
:101670001FE000000010024000004242800442428D
:101680000070004000200C490866FFF7C5FB0546C6
:1016900006E0FFF7C1FB401B022801D9032014E636
:1016A0000648006800F000700028F2D101E0012037
:1016B0000BE6002009E60000000042420010024054
:1016C000042808D14FF0E021096941F004014FF0EE
:1016D000E022116107E04FF0E021096921F00401E7
:1016E0004FF0E02211617047704770B504462546FF
:1016F000681EB0F1807F01D301200FE0681E4FF01B
:10170000E02148610F214FF0FF3001F095F90020F2
:101710004FF0E021886107200861002070BD10B5FE
:10172000FFF7E2FF10BD10B504460CB9012010BD53
:1017300094F83D0028B9002084F83C00204600F0D1
:101740000DF8022084F83D00211D206801F0B2FC54
:10175000012084F83D000020E9E7000008B5016899
:10176000B1F1804F0DD100BF0649C96941F00101B7
:10177000044AD1611146C96901F00101009100BF1D
:1017800000BF08BD0010024001460868C06840F074
:1017900001000A68D0600868006840F001000A682B
:1017A00010600020704701460868C06820F0010002
:1017B0000A68D06000BF0868006A41F21112104048
:1017C00050B90868006A9210104028B9086800688B
:1017D00020F001000A68106000BF0020704770B55B
:1017E0000446002520684069C0F3C01594F839000C
:1017F00021280ED16DB12068406920F08000216859
:101800004861206B10B1206BFEF7A8FF204601F065
:1018100007FD20684069C0F3801594F83A0022283B
:101820000ED16DB12068406920F040002168486108
:10183000606B10B1606BFEF791FF204601F0D0FCA9
:10184000002070BD704701460022002391F8392026
:1018500091F83A3042EA0300704700002DE9F04762
:101860000446206805682068C668206847694FF00C
:101870000008C14605F00F08B8F1000F0AD105F0C5
:10188000200038B106F0200020B1204601F014FD00
:10189000BDE8F087B8F1000F6DD007F0010018B96E
:1018A00006F49070002866D005F0010030B106F40F
:1018B000807018B1E06B40F00100E06305F00400B7
:1018C00030B107F0010018B1E06B40F00200E063B6
:1018D00005F0020030B107F0010018B1E06B40F0F4
:1018E0000400E06305F0080030B107F0010018B112
:1018F000E06B40F00800E063E06B68B305F02000A7
:1019000028B106F0200010B1204601F0D5FC206877
:101910004069C0F38019E06B00F0080010B9B9F11C
:10192000000F22D0204601F05BFC2068406900F0E7
:101930004000B0B12068406920F040002168486153
:10194000606B50B11748616B4863606BFEF724FF12
:1019500010B1606B416B88470CE02046FFF772FFC7
:1019600008E02046FFF76EFF04E02046FFF76AFF1D
:101970000020E0638CE705F0800030B106F08000C5
:1019800018B1204601F0D0FD82E705F0400030B1EB
:1019900006F0400018B1204601F032FC78E700BFA5
:1019A00076E700002931000810B504460CB9012083
:1019B00010BDA06900B100E000BF94F8390028B95B
:1019C000002084F83800204600F028F8242084F80D
:1019D00039002068C06820F400502168C8602046A3
:1019E00001F0BEFC2068006920F490402168086185
:1019F0002068406920F02A00216848612068C0689A
:101A000040F400502168C8600020E063202084F882
:101A1000390084F83A000020CAE7000010B586B00B
:101A200004466F492068884277D100BF6D488069BD
:101A300040F004006B4988610846806900F00400AA
:101A4000019000BF00BF00BF0846C06940F40030ED
:101A5000C8610846C06900F40030019000BF00BFB3
:101A6000042002900220039003200590012004909E
:101A700002A95D48FFF73CF808200290002003907F
:101A800002A95948FFF734F82620FFF757FA032236
:101A900011462620FFF75FFA544855490860002098
:101AA00048600021524881608021C16000210161AD
:101AB000416181614FF40051C161FEF793FF18B19C
:101AC000AB214CA001F078FE00BF4948606344623E
:101AD00000BF464814304D4908601020486000217E
:101AE0004A4881608021C1600021016141618161BA
:101AF000C161FEF777FF18B1BB213EA001F05CFE8B
:101B000000BF42482063446200BF032211462620E2
:101B1000FFF721FA2620FFF711FA3D492068884295
:101B20005CD100BF2F48806940F008002D498861D2
:101B30000846806900F00800019000BF00BF00BFA8
:101B40000846806940F0100088610846806900F00E
:101B50001000019000BF00BF00BF0846C06940F4FC
:101B60008020C8610846C06900F48020019000BF51
:101B700000BF08150290022003900120049003206A
:101B8000059002A92348FEF7B3FF4FF400600290CE
:101B90000020039002A91F48FEF7AAFF4FF400504F
:101BA000029001200390002004900320059002A9D8
:101BB0001948FEF79DFF19480068C06840F02000F2
:101BC00016490968C8602720FFF7B8F902221146B4
:101BD0002720FFF7C0F9002001F0E2FD06B010BD9C
:101BE0000044004000100240000801406C00024028
:101BF000400500202E2E5C53595354454D5C5573BF
:101C00006172745C75736172742E6300FC04002051
:101C100000480040000C014000100140BC040020BE
:101C200077B581B00446154694F83A00202850D183
:101C3000029800B115B9012004B070BD00BF94F83E
:101C40003800012801D10220F6E7012084F838008D
:101C500000BF0298A062A5850020E063222084F8DE
:101C60003A001D48616B88621C48616BC8621C4861
:101C7000616B08630020616B486302AE32682368C1
:101C8000191D2B46606BFEF7E5FE00BF002000909B
:101C900020680068009020684068009000BF00BF86
:101CA00000BF002084F8380000BF2068C06840F4FE
:101CB00080702168C8602068406940F00100216898
:101CC00048612068406940F0400021684861002078
:101CD000B2E70220B0E700008D310008D3310008E0
:101CE0003D31000810B5034693F83A0020282FD163
:101CF00001B10AB9012010BD00BF93F838000128D6
:101D000001D10220F7E7012083F8380000BF996273
:101D10009A85DA850020D863222083F83A0000BF34
:101D2000002083F8380000BF1868C06840F4807055
:101D30001C68E0601868406940F001001C68606140
:101D40001868C06840F020001C68E0600020D2E7FE
:101D50000220D0E710B504462749206888420ED1FA
:101D6000012001F01DFD962002F074FE23A001F079
:101D700025FD962002F06EFE002001F011FD2149A4
:101D80002068884236D12048008800F4004088BB93
:101D90001D48008800F4804070B11C4800780A2873
:101DA00003D000201849088024E01748008840F438
:101DB0000040154908801DE0144800780D2806D120
:101DC0001148008840F480400F49088012E00F4815
:101DD00000780D490988C1F30D010D4A50540A4895
:101DE0000088401C0849088008460088C72801DD93
:101DF0000020088010BD000000440040696E74653A
:101E0000720000000048004016000020180000206A
:101E1000B403002070472DE9F84304460D461646EA
:101E20001F464FF0000994F8390020285CD105B115
:101E300016B90120BDE8F88300BF94F838000128E6
:101E400001D10220F6E7012084F8380000BF00200D
:101E5000E063212084F83900FEF7DEFF8146A68486
:101E6000E6842BE0E08C401EE084A068B0F5805F43
:101E700016D14B46002280212046009701F088FBB6
:101E800008B10320D6E7A846B8F80000C0F3080060
:101E900021684860206908B9AD1C0FE06D1C0DE099
:101EA0004B46002280212046009701F071FB08B1CB
:101EB0000320BFE715F8010B21684860E08C00287B
:101EC000D0D14B46002240212046009701F060FB14
:101ED00008B10320AEE7202084F8390000BF0020BD
:101EE00084F8380000BFA5E70220A3E7704700BFD1
:101EF000FEE7000010B500200F4908600F48006899
:101F000020F070400D4908600846006840F04050DD
:101F1000086000200A49C1F89C01022002F09AFDE5
:101F2000012005490860022002F094FD00200449C8
:101F3000C1F8980110BD000098812142000C0140B9
:101F40000080214200B585B000BF1E48806940F086
:101F500008001C4988610846806900F0080000906C
:101F600000BF00BF00BF0846806940F010008861D4
:101F70000846806900F01000009000BF00BFC0203C
:101F800001900120029003900320049001A90E48C3
:101F9000FEF7AEFD4FF40070019001200290039017
:101FA0000320049001A90948FEF7A2FD0120084979
:101FB00008600849C1F8980100200749086005B089
:101FC00000BD000000100240000C01400010014064
:101FD0009C812142008021422401224210B5002030
:101FE0000F4908600F48006820F070400D490860F4
:101FF0000846006840F04050086001200A49C1F8D6
:102000009C01022002F026FD012005490860022003
:1020100002F020FD00200449C1F8980110BD000025
:1020200098812142000C01400080214270B5054694
:1020300000241748006820F07040154908600846E1
:10204000006840F000400860002616E000201149BA
:102050000860022002F0FEFC01200F49C1F898013F
:102060006006040E0B487C38006808B1601CC4B2DE
:10207000012002F0EFFC701CC6B2082EE6DB15B999
:10208000FFF7ACFF01E0FFF735FF204670BD000011
:10209000000C0140988121420080214270B5044625
:1020A0001548006820F07040134908600846006831
:1020B00040F040500860002010490860002517E0FB
:1020C000E0090E49091D08606006040E022002F0B6
:1020D000C1FC01200A49C1F89801022002F0BAFCB3
:1020E000002006490860022002F0B4FC681CC5B25A
:1020F000082DE5DB70BD0000000C014098812142F5
:102100000080214210B50F48006820F070400D4952
:1021100008600846006840F04050086001200A4905
:1021200008600A49C1F89801042002F093FC0020DD
:1021300005490860042002F08DFC00200349C1F825
:10214000980110BD000C01409C8121420080214279
:1021500010B50F48006820F070400D49086008462F
:10216000006840F04050086000200A4908600A49B1
:10217000C1F89C01042002F06DFC012005490860B3
:102180000549C1F89C01042002F064FC10BD000068
:10219000000C0140988121420080214210B50024AA
:1021A0001448006820F07040124908600846006832
:1021B00040F00040086001200F49086002F04AFC2E
:1021C00001200E49C1F8980102F044FC07E0601CB0
:1021D000C4B2FA2C03DDFFF7BBFF012010BD064897
:1021E000803800680028F2D10349091F086000BF49
:1021F000F4E70000000C01409C8121420080214254
:102200000146CA1701EB92729210A1EB820292B9B9
:10221000642091FBF0F200FB121050B94FF4C8702B
:1022200091FBF0F200FB121008B90120704700206A
:10223000FCE70120FAE70020F8E7000000B585B0D0
:1022400000BF1548806940F01000134988610846B6
:10225000806900F01000009000BF00BF03200190D3
:102260000120029003900320049001A90B48FEF77F
:102270003FFC022001900120029003900320049073
:1022800001A90748FEF734FC002201210348FEF7AC
:10229000BDFD05B000BD000000100240001001406F
:1022A000000C014010B50446204600F08DF82820AF
:1022B00004F0F2F8206028212068FDF75EFF206816
:1022C00044622079216808702E49206806F0DCF805
:1022D0000020C4F89C00C4F8A000C4F8A4000120A9
:1022E000C4F8AC004FF47A70A4F890000121932058
:1022F0000155922001559820045123499420015101
:1023000004F1900007F08AF804F1900007F0C8F893
:1023100004F1900007F0A8F8A089216808812268DC
:10232000111DA06801F094F9B8B1012001F038FA4C
:10233000962002F08FFB15A0D4E9021201F03EFABC
:10234000962002F087FB002001F02AFAB4F8A820BA
:1023500091B2206806F060F810E0012001F020FA48
:10236000962002F077FB10A0D4E9021201F026FAC1
:10237000962002F06FFB002001F012FA082084F88A
:10238000B00010BD19760008797F00085443503A18
:1023900020436F6E6E65637420746F206970202512
:1023A000733A25640D0A00005443503A20436F6E7F
:1023B0006E65637420746F20646F6D61696E202593
:1023C000733A25640D0A000010B504462068B0B1C8
:1023D000012001F0E5F9962002F03CFB0AA001F093
:1023E000EDF9962002F036FB002001F0D9F92068C3
:1023F00006F032F8206802F075FC0020206004F13D
:10240000900007F04DF810BD46726565206D656D52
:102410006F72790D0A0000002DE9F04704468846E6
:1024200016461F46DDE9089A012001F0B9F9962009
:1024300002F010FB3BA001F0C1F9962002F00AFB6C
:10244000002001F0ADF9242104F15800FDF795FEBC
:102450004046FDF7C5FE0546681C04F01DF8A06562
:10246000691CA06DFDF789FE4146A06DFDF7DAFEFF
:102470000020A16D48553046FDF7B2FE0546681CA8
:1024800004F00AF8E065691CE06DFDF776FE314660
:10249000E06DFDF7C7FE0021E06D41553846FDF7C0
:1024A0009FFE0546681C03F0F7FF2066691C206E3E
:1024B000FDF763FE3946206EFDF7B4FE0021206E65
:1024C0004155C4F86C90C4F878A04FF4806003F0D4
:1024D000E3FF20624FF48061206AFDF74EFE4FF467
:1024E0008061A162084603F0D7FF60624FF480610B
:1024F000606AFDF742FE4FF48061E16204F158002A
:10250000E06100216186A08D82B204F13800616A29
:1025100004F092FF4FF4006104F1B40000F05AFBA4
:10252000BDE8F0874D5154545F496E6974436C693E
:10253000656E740D0A0000002DE9F04104460E4658
:1025400017469846012001F02BF9962002F082FAF6
:1025500012A001F033F9962002F07CFA002001F07D
:102560001FF9D0212046FDF708FE3046FDF738FE62
:102570000546681C03F090FFA060691CA068FDF789
:10258000FCFD3146A068FDF74DFE0020A1684855CE
:10259000E76084F80480BDE8F08100004D51545498
:1025A0005F496E6974436F6E6E656374696F6E0D1B
:1025B0000A000000C0F88C107047C1677047C0F86F
:1025C00088107047C0F880107047C0F884107047BA
:1025D0002DE9F043ADF2144D04460D4616461F4654
:1025E000DDF83494DDF8308404F14C003B4632468B
:1025F0002946CDE900890290143804F06EFF60632B
:10260000606B808898B9012001F0CAF8962002F02A
:1026100021FA2DA001F0D2F8962002F01BFA00203A
:1026200001F0BEF800200DF2144DBDE8F08301204A
:1026300001F0B6F8962002F00DFAD4E93123606B70
:10264000818829A001F0BAF8962002F003FA002050
:1026500001F0A6F829E0012001F0A2F8962002F08E
:10266000F9F92FA001F0AAF8962002F0F3F9002062
:1026700001F096F84FF4806304AA05A904F1B400B0
:1026800000F09AFA401C80B9012001F089F89620E8
:1026900002F0E0F927A001F091F8962002F0DAF9B3
:1026A000002001F07DF80020BDE7606B82880168A2
:1026B00004F1B40000F0A7FA401C0028CBD020465B
:1026C00000F048F80120AEE74D5154543A205175BE
:1026D0006575696E67207075626C697368206661E4
:1026E000696C65640D0A00004D5154543A207175AF
:1026F0006575696E67207075626C6973682C206CF3
:10270000656E6774683A2025642C2071756575655F
:102710002073697A652825642F2564290D0A000035
:102720004D5154543A2051756575652066756C6C31
:102730000D0A00004D5154543A20536572696F756B
:102740007320627566666572206572726F720D0A1B
:102750000000000010B5ADF5826D0446012001F0C7
:102760001FF8962002F076F994F8B01051A001F00D
:1027700025F8962002F06EF9002001F011F814B946
:102780000DF5826D10BD94F8B000062806D007281C
:1027900005D009287ED00F2800D118E086E0204619
:1027A000FFF780FD012000F0FBFF962002F052F9B8
:1027B00046A0D4E9021201F001F8962002F04AF98D
:1027C000002000F0EDFF082084F8B0006EE001204A
:1027D00000F0E6FF962002F03DF943A000F0EEFF86
:1027E000962002F037F9002000F0DAFF04F1B4007F
:1027F00000F001FA10B9D4F8A80000B156E04FF487
:10280000806303AA04A904F1B40000F0D5F90028FC
:1028100044D1012000F0C4FF962002F01BF9BDF85E
:102820000C20354935A000F0C9FF962002F012F9BE
:10283000002000F0B5FF04A804F044FD2065BDF8B9
:102840000C1004A804F042FC4C2108530520C4F8E5
:10285000A800BDF80C00ADF8040004A80290012007
:1028600000F09EFF962002F0F5F84C20025B27A0B6
:10287000216D00F0A3FF962002F0ECF8002000F09C
:102880008FFFB4F8A8108BB22068DDE9011205F0C3
:102890002BFE00E003E00021616307E006E0204634
:1028A000FFF792FD204600F043F800BF00BF00BFD5
:1028B00066E700004D515454205441534B3A207365
:1028C000746174653A2025640A0000005443503A4C
:1028D000205265636F6E6E65637420746F3A2025B5
:1028E000733A25640D0A00004D515454205441534D
:1028F0004B20444154410A0078A1000825732C2044
:10290000646174614C656E3A25640A004D515454FB
:102910003A2053656E64696E672C20747970653A4D
:102920002025642C2069643A20253034580D0A0093
:1029300010B5044604B910BDA06820B1A06802F02B
:10294000D1F90020A060206E20B1206E02F0CAF9FB
:1029500000212166A06D20B1A06D02F0C3F9002016
:10296000A065E06D20B1E06D02F0BCF90021E165E9
:10297000206A20B1206A02F0B5F900212162606A64
:1029800020B1606A02F0AEF900216162D4F8B400AF
:1029900030B1D4F8B40002F0A5F90020C4F8B400B6
:1029A000012000F0FDFE962002F054F808A000F08F
:1029B00005FF962002F04EF8002000F0F1FED4F85A
:1029C0008C0018B12046D4F88C10884700BFB2E7BD
:1029D0006D71747420657869743A0A0008B500BF97
:1029E0000E48406940F001000C49486108464069C2
:1029F00000F00100009000BF00BF0322114610202C
:102A0000FEF7A9FA1020FEF799FA002211461120CC
:102A1000FEF7A1FA1120FEF791FA08BD001002405E
:102A200000BFFEE77047000002480068C0F30220C4
:102A3000704700000CED00E010B5002807DA0A0727
:102A4000140E054A00F00F031B1FD45403E00A07BD
:102A5000130E024A135410BD18ED00E000E400E02C
:102A60002DE9F04107460C46164602257E213846E0
:102A700000F011F9401C10B9E81EBDE8F0812FE00C
:102A800020787D2804D07E2803D07F281AD101E049
:102A900000BF00BF7D21384600F0FDF8401C10B992
:102AA0004FF0FF30E9E714F8012B82F0200138469F
:102AB00000F0F1F8401C10B94FF0FF30DDE7A81C22
:102AC00085B20CE014F8011B384600F0E4F8401C15
:102AD00010B94FF0FF30D0E7681C85B200BF00BFCF
:102AE000301EA6F101010EB2CAD17F21384600F096
:102AF000D2F8401C10B94FF0FF30BEE728B2BCE757
:102B000010B504462260A3800020E080E1602072BE
:102B100010BD70B504460D467D2D04D07E2D05D028
:102B20007F2D10D108E0012020721FE00020E080FE
:102B300020720120607219E0E06808B1E068804707
:102B40000020607270BD607A00B90FE0207A18B181
:102B500085F0200500202072E088A188884204DAF0
:102B6000E188481CE0802068455400BF00BFFF207A
:102B7000E8E7F0B585B006460C4615461F463B46CD
:102B8000224600216846FFF7BBFF0BE09DF81010BE
:102B90006846FFF7BEFF28B9BDF806002880002070
:102BA00005B0F0BD04A9304600F04CF80028EDD087
:102BB0004FF0FF30F4E770472DE9F04104460D4631
:102BC00016461F463B4632462946201DFFF7D1FFD9
:102BD000BDE8F08170B504460D46284603F05CFC64
:102BE000206029462068FDF7C8FA2A46201D216882
:102BF00000F041F870BD01460869002801DC0120A1
:102C000070470020FCE770B504460E4615462AB210
:102C10003146201DFFF724FF70BD000008B50849AC
:102C20000968C9084FF47A72B1FBF2F1414300918F
:102C300000BF00BF00994A1E00920029F9D108BDCB
:102C4000600100200246D068002802DC4FF0FF300F
:102C50007047D068401ED0605068431C53600378B2
:102C60000B701369106818445368984201D81068B3
:102C700050600020ECE7034613B109B1022A02DAE2
:102C80004FF0FF3070479960596019600020D8609C
:102C90001A6100BFF6E70246D0681369984202DB6A
:102CA0004FF0FF307047D068401CD0609068431CE4
:102CB000936001701369106818449368984201D8B2
:102CC000106890600020EDE770B500260024002514
:102CD0003A4806683604001D006806443848B6FBCA
:102CE000F0F438480088A0423AD036490C8040F2CF
:102CF000B2750EE02846FFF783FA30B1B4F5B77F1E
:102D000002D3A4F5B77402E006E0A4F26D14681CC7
:102D100085B2B4F5B67FEDD800BF2B48858000257D
:102D200016E029498888FFF76BFA30B1012D04D1EC
:102D30001D2C01D31D3C09E00CE02448405DA0425D
:102D400003D82248405D241A00E003E0681C85B2E5
:102D50001C2CE6D200BF681C1B498871601CC8711E
:102D60001748B6FBF0F100FB11644FF46160B4FB4F
:102D7000F0F0154908704FF46160B4FBF0F100FB0E
:102D800011403C21B0FBF1F00F4948704FF46160F5
:102D9000B4FBF0F100FB11403C21B0FBF1F201FB70
:102DA0001200094988700B46DA799979988800F001
:102DB0000FF805490872002070BD00001828004077
:102DC0008051010030000020D8050020CC9F000871
:102DD000F0B503460C461546642093FBF0F0C6B2EE
:102DE000642093FBF0F700FB1730C1B2132E02DD15
:102DF00001F16400C1B20846CF1701EB977701EBF0
:102E0000A707BAB2072092FBF0F700FB172082B2A7
:102E10005719601EDFF82CC01CF80000384482B23D
:102E2000CF1701EB9777BF10A1EB87071FB9032CD2
:102E300001DA501E82B2072092FBF0F700FB172048
:102E4000C0B2F0BDC09F000810B5114800684068CE
:102E500000F0010030B16FF001000D4909684860D1
:102E6000FFF732FF0A480068406800F0010048B1EF
:102E70006FF00200064909684860FFF725FF05A0CA
:102E800000F09CFC6FF0040001490968486010BD27
:102E9000C4050020414C41524D2041210D0A000043
:102EA000704730B58FB0054600240120059000041E
:102EB00006900020079002200C90C1030D910E9502
:102EC00005A8FEF7DDF904460CB100BFFEE70F20B0
:102ED000009002200190002002904FF48060039047
:102EE0000020049002216846FEF788F804460CB1E1
:102EF00000BFFEE70FB030BD10B5FDF793FFFEF742
:102F00000EFC10BD1148006840F001000F49086038
:102F1000084640680E4908400C4948600846006869
:102F20000C490840094908600846006820F48020E0
:102F300008600846406820F4FE0048604FF41F0017
:102F40008860C80304490860704700000010024010
:102F50000000FFF8FFFFF6FE08ED00E010B51E4888
:102F60000068C06800F0010080B31C480068406839
:102F700030B11A4A12689068184A12685168884736
:102F800005F0DCFA044615480068406820601348E4
:102F9000006880686060204600F0FEFE0F48006810
:102FA000807808B906F048FE00200B49096848629D
:102FB00000BF0A480068008807490968C8620748D6
:102FC000006801880448C16000BF00BF6FF00100C5
:102FD00001490968086110BDA8120020AC01002059
:102FE00010B515480068C06800F00100F0B105F0A8
:102FF000A5FA044611480068206000206060204661
:1030000000F0CAFE0E48007808B906F063FE002002
:1030100009490968486200BF4FF47A700649096897
:10302000C86201460448C16000BF00BF6FF00100E4
:1030300001490968086110BD8405002028000020AE
:103040002400002010B519480068C06800F0010095
:1030500028B305F073FA04461548006840682060FC
:103060001348006880686060204600F095FE1048B4
:103070000068807808B906F075FE00200B490968E1
:10308000486200BF0A480068008808490968C862A9
:103090000748006801880548C16000BF00BF6FF0A5
:1030A000010002490968086110BD0000E812002013
:1030B000B001002000220268184B984208D0B0F1FD
:1030C000804F05D0164B984202D0164B984203D140
:1030D00022F070024B681A43104B984208D0B0F1AE
:1030E000804F05D00E4B984202D00E4B984203D130
:1030F00022F44072CB681A4322F080024B691A43D3
:1031000002608B68C3620B688362044B984201D1F2
:103110000B6903630123436170470000002C0140E9
:10312000000400400008004070B505466C6A0020AD
:10313000E085E0842046FEF785FB70BD70B506464D
:103140000025746A20684069C0F3C01594F83900FE
:10315000212805D125B10020E084204600F060F848
:1031600020684069C0F3801594F83A00222805D100
:1031700025B10020E085204600F032F8E06B40F0F9
:103180001000E0632046FEF75DFB70BD70B505469C
:103190006C6A2868006800F02000B0B90020E08563
:1031A0002068C06820F480702168C8602068406989
:1031B00020F00100216848612068406920F040004B
:1031C00021684861202084F83A002046FEF7C2FDBD
:1031D00070BD70B50446656A2846FEF71BFE70BDDB
:1031E0000168C96821F490710268D1600168496979
:1031F00021F0010102685161202180F83A107047E6
:1032000010B504462068C06820F040002168C860FE
:10321000202084F839002046FEF768FE002010BD0B
:103220000168C96821F0C0010268D160202180F8DE
:1032300039107047F8B504462068006800F01000A7
:1032400010282BD100BF002000902068006800905B
:1032500020684068009000BF00BF2046FEF7BFFA1C
:1032600020680668206846680D4800684668C6F50C
:10327000FA700C4908800CA10D48FCF789FF05463F
:103280001DB101200B49087001E000F00DFA4FF468
:10329000FA7207492046FEF7C3FC00BFF8BD0000E4
:1032A0004005002014000020444F4E45000000005F
:1032B000C00100201900002070B5044694F83A00BF
:1032C00022284AD1A068B0F5805F13D1A56A206991
:1032D00040B920684068C0F308002880A06A801CBC
:1032E000A06219E020684068C0B22880A06A401C33
:1032F000A06211E0206938B920684068C1B2A26AB2
:10330000501CA062117007E02068406800F07F0147
:10331000A26A501CA0621170E08D401E80B2E08550
:10332000C8B92068C06820F020002168C860206803
:10333000C06820F480702168C8602068406920F06F
:10334000010021684861202084F83A002046FEF7F9
:1033500001FD002070BD0020FCE70220FAE700001C
:103360002DE9F041044600252068006920F4405012
:10337000E1680843216808612169A0680843616920
:10338000084305432068C06841F20C618843284324
:103390002168C8602068406920F44070A169084332
:1033A000216848615F49206888425CD1FDF70EFFC3
:1033B00000EBC00101EB001061688900B0FBF1F681
:1033C000FDF704FF00EBC00101EB0010616889000C
:1033D000B0FBF1F06421B0FBF1F000EBC00101EBB8
:1033E0000010A6EB8000322101EB00106421B0FB3D
:1033F000F1F000F0F006FDF7E9FE00EBC00101EB93
:10340000001061688900B0FBF1F06421B0FBF1F0BD
:1034100006EB0016FDF7DAFE00EBC00101EB001031
:1034200061688900B0FBF1F7FDF7D0FE00EBC00149
:1034300001EB001061688900B0FBF1F06421B0FB82
:10344000F1F000EBC00101EB0010A7EB800032218E
:1034500001EB00106421B0FBF1F000F00F003044EC
:10346000216888605BE0FDF7A1FE00EBC00101EB85
:10347000001061688900B0FBF1F6FDF797FE00EBE4
:10348000C00101EB001061688900B0FBF1F064211C
:10349000B0FBF1F000EBC00101EB0010A6EB8000E7
:1034A000322101EB00106421B0FBF1F000F0F006D6
:1034B000FDF77CFE00EBC00101EB001061688900A4
:1034C000B0FBF1F06421B0FBF1F006EB0016FDF764
:1034D0006DFE00EBC00101EB001061688900B0FBDC
:1034E000F1F7FDF763FE00EBC00101EB001061682E
:1034F0008900B0FBF1F06421B0FBF1F000EBC001FA
:1035000001EB0010A7EB8000322101EB00106421D9
:10351000B0FBF1F000F00F00304421688860BDE896
:10352000F081000000380140014691F8390021285F
:103530002CD18868B0F5805F0FD10A6A1088C0F37B
:1035400008000B685860086918B9086A801C08628E
:1035500009E0086A401C086205E00B6A581C086212
:1035600018780B685860C88C401E80B2C88458B95F
:103570000868C06820F080000B68D8600868C068E0
:1035800040F040000B68D860002070470220FCE744
:103590002DE9F04104460D4617469846069E21E067
:1035A000701CF8B12EB1FDF737FCA0EB0800B0425B
:1035B00018D92068C06820F4D0702168C8602068DD
:1035C000406920F0010021684861202084F839001A
:1035D00084F83A0000BF002084F8380000BF0320C0
:1035E000BDE8F081206800682840A84201D1012090
:1035F00000E00020B842D3D00020F1E710B5034826
:10360000FFF718FE0148FEF729F910BD7C040020E1
:1036100010B500240C48FEF721F900BF01E0641C3E
:1036200000BF0948FEF70FF92028F8D100BF002499
:1036300001E0641C00BF012204490348FEF752FB6D
:103640000028F6D100BF10BDBC04002018000020E7
:1036500070B504460D46264600211FE0002315E004
:103660003278761C302A08DB392A06DC03EB83002B
:103670004300A2F13000034408E0032901DA2E2AB6
:1036800001D0032900D102E0002070BDE8E700BFAF
:10369000FF2B01DD0020F8E76B54491C0429DDDB1A
:1036A0000120F2E700BFFEE710B5012000F078F836
:1036B000962001F0CFF91D4802881D491DA000F099
:1036C0007DF8962001F0C6F9002000F069F804F0BA
:1036D00035FF04461F490968086814490A88521CC6
:1036E0001349FCF72FFD00211A48006800680F4AB3
:1036F000128881540D480088401C1649096888804A
:1037000015482060134800686060204600F044FBC4
:1037100000200649088000BF03E00021044A11543C
:10372000401CB0F5FA7FF8DB10BD0000140000204B
:10373000C001002053494D373630303D3D3D3D3EC0
:103740004D43553A25732C206C656E3A25640D0A5D
:10375000000000001C0000200565000870B504464C
:103760000D4642F210732A4621460248FEF753FBEB
:1037700070BD00007C04002010B50446012000F05C
:103780000FF84FF47A7001F065F9204600F016F852
:10379000962001F05FF9002000F002F810BD000053
:1037A000014619B90022034B1A6002E00122014BC5
:1037B0001A607047B401224200BFFEE70FB4054B08
:1037C00010B503A9044A029800F030F810BC5DF867
:1037D00014FB0000C94C0008100000200FB4084B77
:1037E00010B504A902AA039800F020F8044602A923
:1037F000002000F04CFA204610BC5DF814FB0000DD
:103800008F3C000800487047BC01002002E008C857
:10381000121F08C1002AFAD170477047002001E04A
:1038200001C1121F002AFBD1704700002DE9FF4F94
:103830008DB00F460546002606E025280BD0DDE9B1
:103840000F1290476D1C761C28780028F5D111B016
:103850003046BDE8F08F0024A246A1460122EC4983
:1038600000E0044315F8013F203B02FA03F0084250
:10387000F7D128782A2810D06FF02F022878A0F1ED
:103880003001092914D80AEB8A0102EB410144F006
:10389000020400EB010A6D1CF0E701CF5FEA000AA9
:1038A00003D544F40054CAF1000A44F002046D1C2C
:1038B00028782E2817D115F8010F44F004042A287F
:1038C0000ED06FF02F022878A0F1300109290AD814
:1038D00009EB890102EB410100EB01096D1CF2E7E4
:1038E00057F8049B6D1C28786C280FD006DC4C28F8
:1038F00017D068280DD06A2814D104E0742810D09D
:103900007A280FD10DE044F400140AE044F4801446
:1039100001E044F440146978814202D104F5801436
:103920006D1C6D1C2A786E2A1FD00CDC632A31D0E6
:1039300004DC002A8BD0582A11D1A3E0642A68D075
:10394000692A0CD165E0732A2ED004DC6F2A73D06B
:10395000702A04D19BE0752A6FD0782A6ED0104669
:10396000DDE90F129047761C50E1C4F302500228A3
:1039700006D0032809D0042801CF09D0066045E10C
:1039800001CFF117C0E9006140E101CF06803DE1C0
:1039900006703BE117F8040B8DF8000000208DF84D
:1039A0000100EB46012003E057F804BB4FF0FF3065
:1039B00061074FF0000102D40DE008F101018846D3
:1039C00049450FDA8045F8DB1BF808100029F4D1CF
:1039D00008E008F1010188468142FADB1BF8081073
:1039E0000029F6D1DDE90F23AAEB08008146214624
:1039F00000F036F9304400EB080604E0DDE90F1270
:103A00001BF8010B9047B8F10108F7D22146484650
:103A1000F7E00A21C4F302534FF0000B0891022B88
:103A200004D001CFC117032B09D00AE0FF1D27F0F6
:103A30000707F7E8020108E032E01FE020E000B2EB
:103A4000C117042B01D140B2C117031E71F100034D
:103A500007DA4FF0000CD0EB0C006CEB01012D23CA
:103A600002E0230504D52B238DF82430012303E045
:103A7000E30701D02023F7E7984658E00A2110E039
:103A800010210EE010204FF0000B08900CE01021E8
:103A90004FF0000B44F004044FF00809089103E0D4
:103AA00008214FF0000B0891C4F30253022B04D0FD
:103AB00001CF0021032B06D006E0FF1D27F00707EA
:103AC000F7E8020103E080B2042B00D1C0B24FF04E
:103AD000000823072BD5702A07D0DDF820C08CF012
:103AE000100C5CEA0B0C05D00EE040238DF824305E
:103AF000012308E050EA010306D030238DF824307A
:103B00008DF8252002239846DDF820C08CF0080CA3
:103B10005CEA0B0C0BD150EA010301D1630706D517
:103B200030238DF824304FF00108A9F10109582AFB
:103B300004D038A20B9208AA0A920BE03AA2F9E745
:103B40005B46089AFCF7A0FB0B9B9B5C0A9A521EF3
:103B50000A92137050EA0102F2D10A98ADEB00000C
:103B600000F1200B600702D524F4803401E04FF00F
:103B70000109D94502DDA9EB0B0000E0002000EBB4
:103B80000B0141440890AAEB010AE00306D4DDE9E9
:103B90000F232146504600F063F806444FF0000919
:103BA00008E009A911F80900DDE90F12904709F1B1
:103BB0000109761CC145F4DBE0030CD5DDE90F23D8
:103BC0002146504600F04CF8064404E0DDE90F12AF
:103BD00030209047761C0899481E08900029F5DC93
:103BE00008E00A980A990078491C0A91DDE90F1249
:103BF0009047761CBBF10001ABF1010BF1DC2146D3
:103C00005046DDE90F2300F019F806446D1C1BE651
:103C100009280100303132333435363738396162A2
:103C20006364656600000000303132333435363766
:103C30003839414243444546000000002DE9F04137
:103C4000044600251E461746880404D405E039467C
:103C50002020B0476D1C641EF9D52846BDE8F081D0
:103C60002DE9F041044600251E469046C80301D5C3
:103C7000302700E02027880404D505E04146384677
:103C8000B0476D1C641EF9D52846BDE8F0810A686E
:103C9000531C0B60107070472DE9F74181B004464A
:103CA000154600260027B0461CB9701E04B0BDE8BA
:103CB000F081D4F80260B4F80080218819480088A7
:103CC000001D08442080208802F0E6FBC4F80200B2
:103CD0002188D4F80200FCF750FAD4F802004246DA
:103CE000314600F089FC0746002000900222694618
:103CF000384600F081FC0746BDF8080004F05AFA87
:103D00000290022202A9384600F076FC07460548D8
:103D1000028829463846FCF715FA304600F0E2FFE3
:103D20000020C3E79C01002030B595B004460D4645
:103D3000402105A8FCF721FA14216846FCF71DFA7A
:103D400021466846FCF76EFA294605A8FCF76AFA90
:103D500005AA69460A48FCF7A2FC401C70B901207C
:103D6000FFF71EFD962000F075FE06A0FFF726FD6A
:103D7000962000F06FFE0020FFF712FD15B030BD59
:103D8000DC0900207772697465206669666F2065BA
:103D900072726F72210D0A0070B506460C2002F097
:103DA0007BFB044614B94FF0FF3070BD002060600B
:103DB000A06026600D48006818B90C480460002017
:103DC000F3E70A480068806810B90848056802E00F
:103DD00006480068856800E0AD68A8680028FBD147
:103DE000AC606560A06000BFDFE70000200000203D
:103DF00010B5024604E01089401C80B210810146D3
:103E00000029F8D09088801C138A984201DD002098
:103E100010BD0B129488601C9080D0680355948864
:103E2000601C9080D06801550846F1E770B50446E3
:103E30000E461546A0882844801C218A884202DD4F
:103E40004FF0FF3070BDC5F30721A288501CA08041
:103E5000E0688154A288501CA080E0688554A28844
:103E6000E16888182A463146FCF76CF9A088284496
:103E7000A080A81CE6E7000010B50446364800788C
:103E800090B90120FFF78CFC962000F0E3FD33A0F1
:103E9000FFF794FC962000F0DDFD0020FFF780FC8A
:103EA00032A005F0CFFB55E02B480078022803D064
:103EB0002948007804284DD12E48006888BB2E4838
:103EC000FCF71DFC002845D12C480078012841D181
:103ED000942002F0E1FA274908600846026814328B
:103EE00001682548FCF7A3FB002833D000202349B4
:103EF000087020480068143005F0A4FB0120FFF78B
:103F00004FFC962000F0A6FD1A48016814311CA051
:103F1000FFF754FC962000F09DFD0020FFF740FCC9
:103F200018E0FFE70120FFF73BFC962000F092FD30
:103F300010480168143112A0FFF740FC962000F0F1
:103F400089FD0020FFF72CFC10480078401C40B28F
:103F50000E490870002010BD50010020737461727A
:103F6000742073656E642041540D0A0041540D0A9B
:103F70000000000054010020DC0900205101002055
:103F800073656E64696E673A257300005E010020F8
:103F90002DE9FE4380460E461B4A07CA8DE80700FE
:103FA0004FF0FF370025344600E0641C207872286B
:103FB000FBD020780A28F8D0002509E05DF825100C
:103FC0002046FCF7E5F808B16FB203E0681CC5B203
:103FD000032DF3D300BF27B1012F06D0022F0CD140
:103FE00007E001200949087008E00120074908702E
:103FF00004E001200549087000E000BF00BF03484D
:10400000007840B2BDE8FE83D89F0008510100202F
:104010002DE9FE4380460E461A4A07CA8DE807007E
:104020004FF0FF370025344600E0641C20780D284F
:10403000FBD020780A28F8D0002509E05DF825108B
:104040002046FCF7A5F808B16FB203E0681CC5B2C2
:10405000032DF3D300BF27B1012F06D0022F09D1C2
:1040600007E001200849087005E0012006490870B2
:1040700001E000E000BF00BF0348007840B2BDE8A7
:10408000FE8300000CA000085101002010B50A4674
:10409000436803610276222A01D04E2A13D104E03C
:1040A0005C2902D143685B1C43604468631C436025
:1040B0000368195D09B12229F2D1046943681B1B09
:1040C0005B1E436119E0302A17D100BFD0E90034EC
:1040D000195D302901DB392903DD2E2901D00021AA
:1040E00002E043685B1C43600029EFD103695B1E5B
:1040F0000361046943681B1B436110BD70B505462D
:104100000C4611480088401E0F490880284601F0DF
:1041100093FEA11C022202FB00100B4949880844AF
:10412000094948800846008860B90848006828B1F5
:10413000064800684988084404490860002002498C
:104140000880488070BD0000980100209401002084
:104150002DE9FE4380460E461A4A07CA8DE807003D
:104160004FF0FF370025344600E0641C20780D280E
:10417000FBD020780A28F8D0002509E05DF825104A
:104180002046FCF705F808B16FB203E0681CC5B221
:10419000032DF3D300BF27B1012F06D0022F09D181
:1041A00004E001200849087005E004E00120064908
:1041B000087000E000BF00BF0348007840B2BDE8CF
:1041C000FE8300005CA00008510100202DE9F04FA3
:1041D00087B00F461822894901A8FBF7B3FF4FF0BB
:1041E000FF3800263C4600E0641C20780D28FBD0F8
:1041F00020780A28F8D000260BE001A850F82610F5
:104200002046FBF7C5FF10B14FFA86F803E0701C9B
:10421000C6B2062EF1D300BFB8F1060F70D2DFE8A8
:1042200008F003426A6B707175A12046FBF7B0FF7E
:10423000044611342046FCF70DF80546B5F57A7FA3
:104240001DDD0120FFF7ACFA962000F003FC2946A3
:1042500070A0FFF7B3FA962000F0FCFB0020FFF7F8
:104260009FFA7448006818B10020724909688847AD
:10427000012071490870801E07B0BDE8F08F6FA162
:104280002046FBF785FF0446A41C6D496D4A128841
:1042900088182A462146FBF755FF6A4800882844BB
:1042A00068490880A0E0684800F06FFC05460DB33F
:1042B0000120FFF775FA962000F0CCFB63A0FFF712
:1042C0007DFA962000F0C6FB0020FFF769FA2988E6
:1042D000686805F0ADFA29886868FFF73FFA6868F2
:1042E00020B1686800F0FEFC00206860284600F0FD
:1042F000F9FC002578E077E001204F49087073E071
:1043000071E071E04FF0000A0FF250190120FFF741
:1043100047FA962000F09EFB494953A0FFF74EFA5A
:10432000962000F097FB0020FFF73AFA49464448F0
:10433000FBF72EFF0446DCB90120FFF731FA962087
:1043400000F088FB21464DA0FFF738FA962000F0D8
:1043500081FB0020FFF724FA3648006818B10020DE
:10436000344909688847012033490870801E83E773
:104370004846FBF735FF00EB040B5846FBF76AFF96
:104380000546C82D1BD00120FFF70AFA962000F041
:1043900061FB29463FA0FFF711FA962000F05AFB77
:1043A0000020FFF7FDF92348006818B100202149DB
:1043B00009688847012020490870801E5CE73AA1FF
:1043C0002046FBF7E5FE00F1040A00201D490880A5
:1043D0000120194908701748006818B1504615495E
:1043E0000968884700BF00BF00BF384600F07AFC6C
:1043F00000271148007840B23EE7000068A000089E
:104400002B434348524543563A20444154412C31B2
:104410002C000000726573706F6E73652073697A8B
:104420006520697320696C6C6567616C3A2564214D
:104430000A00000048000020510100200D0A000081
:10444000F40500205A010020DC09002073656E6429
:10445000696E672E2E2E2E2E0A00000048545450EE
:104460002F312E3100000000687474702072656373
:10447000656976653A25730A00000000496E766129
:104480006C69642076657273696F6E20696E202591
:10449000730D0A00496E76616C69642073746174EF
:1044A00075733A25640D0A000D0A0D0A000000001C
:1044B00070B504460D4616460120FFF771F99620A7
:1044C00000F0C8FA0CA0FFF779F9962000F0C2FAC4
:1044D0000020FFF765F904EB44000D4901EB800073
:1044E000806838B104EB440001EB800031468268FB
:1044F0002846904770BD000073656E64207061634C
:104500006B61676520746F206465766963650A0076
:10451000B00F002070B504460D46164604EB44006B
:10452000064901EB8000406838B104EB440001EB20
:104530008000314642682846904770BDB00F002089
:104540000146302905DB392903DCA1F13002D0B264
:1045500002E0A1F15702D0B27047000010B5044646
:1045600010220D4904F10900FBF74FFE88B101202C
:10457000FFF716F9962000F06DFA08A0FFF71EF974
:10458000962000F067FA0020FFF70AF94FF0FF309D
:1045900010BD0020FCE7000024110020546F6B6563
:1045A0006E206572726F722E0A0000002DE9FC41C8
:1045B00004460D4617464FF000083A212046FBF707
:1045C00005FEB0F1000802D1401EBDE8FC81A8EB59
:1045D0000406324621462846FBF7ECFD0020A8558C
:1045E000082208F101016846FBF7E4FD6846FBF785
:1045F00031FE38600020E8E770B504460E461546E7
:104600002A4631462046FBF79DFD2C44204670BDCE
:104610002DE9FE4380460E461C4A07CA8DE8070076
:104620004FF0FF370025344600E0641C20787228E4
:10463000FBD020780A28F8D0002509E05DF8251085
:104640002046FBF7A5FD08B16FB203E0681CC5B2B8
:10465000032DF3D300BF27B1012F06D0022F0ED1B7
:1046600004E001200A4908700AE009E009A1204697
:10467000FBF78EFD10B101200549087000E000BF76
:1046800000BF0348007840B2BDE8FE83E49F000805
:1046900051010020524541445900000010B5044624
:1046A0000321204600F002F810BD00002DE9F04182
:1046B00007460E4600240025062001F0EDFE0446C4
:1046C00000202060A0800C202080208801F0E4FEE3
:1046D000C4F802002188D4F80200FBF74EFDD4F89C
:1046E0000250012E09D116488068401C1449886088
:1046F000886803F06BFDA8600AE0022E08D110481C
:104700000068401C0E490860086803F05FFDA8605F
:10471000032E08D10A484068401C0949486048688F
:1047200003F054FDA860384603F044FDE8803420CF
:104730002870304603F03EFD68802046BDE8F081D9
:104740003411002010B5012001F0A6FE044600201F
:104750002070204610BD000010B5002400200A493A
:1047600008808020094908800846008801F094FEEE
:1047700004460CB9002010BD002020800220024910
:1047800008802046F7E700009C0100209E010020E1
:104790002DE9FE4380460E462B4A07CA8DE80700E6
:1047A0004FF0FF370025344600E0641C20780D28C8
:1047B000FBD020780A28F8D0002509E05DF8251004
:1047C0002046FBF7E5FC08B16FB203E0681CC5B2F8
:1047D000032DF3D300BF27B1012F10D0022F2BD10F
:1047E00011E01AA12046FBF7D3FC0446A01DFBF7FD
:1047F00031FD184908700120174908701DE001209B
:104800001549087019E00120FEF7CAFF962000F054
:1048100021F9214611A0FEF7D1FF962000F01AF9E8
:104820000020FEF7BDFFE01DFBF714FD09490870ED
:1048300001200949087000E000BF00BF0648007869
:1048400040B2BDE8FE830000F09F00082B435351A7
:104850003A2000004C000020510100206373713A9F
:1048600025730D0A0000000070B5044625462E6829
:104870000EA12868FBF78CFCB0B10FA12868FBF7EC
:1048800087FC0646361D3046FBF7F1FCA0800CA1E4
:104890003046FBF77DFC0646B61CA28831462868E8
:1048A000FBF750FC012070BD0020FCE75245435649
:1048B0002046524F4D3A00002B4950440000000062
:1048C0000D0A00007CB505466946284600F0ACFAA2
:1048D0000646BDF802004FF6F871884211D101205A
:1048E000FEF75EFF962000F0B5F81DA0FEF766FF0C
:1048F000962000F0AFF80020FEF752FF04F0AEFE65
:104900002CE00120FEF74CFF962000F0A3F8BDF844
:10491000021019A0FEF752FF962000F09BF800202D
:10492000FEF73EFFBDF80210C8B200F051F9044690
:104930007CB90120FEF734FF962000F08BF814A01C
:10494000FEF73CFF962000F085F80020FEF728FFD8
:104950007CBD606810B130466168884700BFF7E7EA
:10496000726563656976652061206765742072658C
:1049700071756573740A00000A526563656976652E
:10498000206120636F6D6D616E643A25640A0000DA
:104990006E6F207375636820636F6D6D616E642048
:1049A00066696E64000000002DE9FC410446D4F8FD
:1049B0000200218847184FF0000800261BE0BDF8D0
:1049C0000210C8B200F01CF9054685B90120FEF7B7
:1049D000E7FE962000F03EF8BDF802100AA0FEF7B0
:1049E000EDFE962000F036F80020FEF7D9FE3046A6
:1049F000A968884700BF6946204600F047FA061EAE
:104A0000DDD1BDE8FC8100006F626A656374205BE4
:104A100025645D206E6F7420666F756E6420696E0C
:104A2000206C6973740A000010B504460420FCF77A
:104A300047FE0148046010BD0C00002030B504465C
:104A4000002504E04FF47A7000F004F86D1CA542D4
:104A5000F8D330BD70B5034600224FF0E0267569EB
:104A60000D4E366803FB06F44FF0E026B16910E006
:104A70004FF0E026B06988420BD0884202D20E1A6D
:104A8000324402E02E1A0E4432440146A24200D3C0
:104A900000E0EDE700BF70BD0C00002010B504463B
:104AA0004CB1D4F8020030B1D4F8020000F01AF989
:104AB0000020C4F80200204600F014F9002410BDC4
:104AC00010B5044614B1204600F00CF910BD10B525
:104AD00004461CB1204600F005F9002410BD10B5B5
:104AE000044604B910BD606820B1606800F0FAF8AF
:104AF00000206060204600F0F5F8002400BFF1E7D8
:104B0000F0B587B004460E461546A8B2ADF81400BD
:104B100005A9304602F086FB0390A8B2ADF8160056
:104B20000DF11601304602F02DFB0490D4F88800F8
:104B300050B1BDF816000090BDF81420DDE9031354
:104B40002046D4F88870B84707B0F0BD10B50446C9
:104B500003F006FC012809D1022006490870064826
:104B600004F09EFC054803F0D5FE01E0002010BDD6
:104B700000BFFCE780010020F4100020354D000844
:104B8000C1680160002181807047014601F5B46071
:104B9000D1F8CC2550F82200704700F5B462D0F867
:104BA000C83542F82310704770B5054607480468B9
:104BB00007E0211D2846FBF71AFB08B9204670BD07
:104BC0002468002CF5D10020F9E70000A80100209E
:104BD0000246002109E0084810F83100904203D154
:104BE000054800EBC1007047491C04480068814239
:104BF000F1DB0020F7E7000040110020A0010020B9
:104C0000024600210CE001EB4100084B13F82000A4
:104C1000904204D101EB410003EB80007047491C36
:104C2000034800688142EEDB0020F7E7C011002056
:104C3000A4010020F0B50C46059E8588E91E7F2959
:104C40002ADD25072D0E02F0010745EAC70503F00E
:104C5000030745EA470506F001073D43C7683D7075
:104C60000D46CF1701EB5767FF11A1EBC717FFB236
:104C700047F08007D0F80CC08CF80170CF1701EB1B
:104C80005767C7F3C717D0F80CC08CF80270CD1C5B
:104C90008580C568056015E025072D0E02F0010727
:104CA00045EAC70503F0030745EA470506F0010793
:104CB0003D43C7687D70C768B9708D1C8580C56825
:104CC0006D1C0560F0BD000000BF054A126802F0CF
:104CD0004002002AF9D0C2B2014B1B1D1A60704776
:104CE0000048004010B5002821D0114B0022001FC1
:104CF000196803E0814203D80A4649680029F9D1BE
:104D000052B11368841A9C4204D1006818441060A0
:104D1000104602E0506000E0186039B102680B1ADA
:104D2000934203D10B681A4402604968416010BD88
:104D3000B401002010B5044616480078012819D0A7
:104D4000022821D1A01C38B9012012490870AFF205
:104D50001B0003F0EDFE0CE0012C07D103200D49F0
:104D60000870AFF22F0003F02FFC02E00A4804F0B5
:104D70007BFB0DE024B9AFF2430003F025FC02E019
:104D8000054804F071FB03E0034804F06DFB00BF2D
:104D900000BF10BD80010020F410002010B50446B3
:104DA0000648408820B9208803F004FA03490880A7
:104DB00002484188A01C084410BD00009801002052
:104DC00070B5044600F008F8054610222946204632
:104DD000FBF7B8F970BD000000487047E4050020FB
:104DE000014890F9000070475001002070B504465A
:104DF0000D46208803F0DEF92880608803F0DAF998
:104E00006880A08803F0D6F9A880201D70BD1CB56D
:104E100004460021009101916946204600F00EF9F8
:104E2000DDE900011CBD00002DE9F04105460C46FE
:104E300055F8020F00F10C062F68B86803F0C6F9A8
:104E40000B498860308803F0B5F92080708803F042
:104E5000B1F96080B08803F0ADF9A080F08803F06C
:104E6000A9F9E08055F802091230BDE8F081000090
:104E70003411002070B5044614B94FF6FF7070BDB0
:104E8000D4F80250688803F095F9F8E72DE9F0416D
:104E900004460D46002600271648006821888842EF
:104EA00004D0144800682188884204DD002011499C
:104EB0000860BDE8F0810F48006858B90D480068E7
:104EC0000C300C490860D4F80270B86803F07EF921
:104ED00009494860D4F8020006490968461805489F
:104EE0000068801D0349086029463046FFF77EFFB1
:104EF000DFE7000094010020341100202DE9F04785
:104F000007460D4614461E464FF000093888288093
:104F1000288803F04FF92880288800F08DFF80460C
:104F2000B8F1010F0BD178882080208803F042F976
:104F300020802288391D3046FBF704F936E02888A6
:104F400000F042F8208007F10209228849463046E5
:104F5000FBF7F8F828880E2826D2DFE800F02507AE
:104F6000141D20190E1E21180D25251FD6E900211C
:104F7000104603F097F918E000BFD6E9002110466B
:104F800003F045F911E0306803F033F90DE000BF9C
:104F9000306803F01BF908E000BF00BF05E000BF68
:104FA000308803F007F900E000BF00BF20883844D4
:104FB000001DB8F1000F01D1012100E00021A0EB9C
:104FC0004100BDE8F087000010B504460E2C1AD24F
:104FD000DFE804F019070B0F130D0910140C081665
:104FE000171100BF00BF082010BD00BF00BF042084
:104FF000FAE700BF00BF0120F6E700BF0220F3E799
:1050000000BF0020F0E70120FEF7CAFB9620FFF763
:1050100021FD05A0FEF7D2FB9620FFF71BFD002027
:10502000FEF7BEFBFF20DFE7556E6B6E6F772064E7
:1050300061746120747970652E0A00007CB50546A4
:105040000C460020019000902846FFF7A7FE064678
:1050500023466A4601A93046FFF750FFBDF800100D
:10506000BDF80400FFF74AF87CBD00002DE9FF41C0
:1050700080460E46264B0FCB8DE80F004FF0FF37D2
:105080000025344600E0641C20780D28FBD02078F1
:105090000A28F8D0002509E05DF825102046FBF726
:1050A00077F808B16FB203E0681CC5B2042DF3D3E2
:1050B00000BF37B1012F0BD0022F0AD0032F1FD111
:1050C0000EE001201349087003201349087018E00E
:1050D00017E001200F49087003200F49087010E005
:1050E0000120FEF75DFB9620FFF7B4FC0BA0FEF756
:1050F00065FB9620FFF7AEFC0020FEF751FB00E0B9
:1051000000BF00BF0348007840B204B0BDE8F081A2
:10511000FC9F000851010020500100204E65740DD5
:105120000A0000002DE9FC4180460E46294903C9CA
:10513000CDE900014FF0FF370025344600E0641C44
:1051400020780D28FBD020780A28F8D02248007853
:10515000D0B90F2221462148FAF7F4FF00201F4959
:10516000C8730120FEF71CFB9620FFF773FC1B4958
:105170001BA0FEF723FB9620FFF76CFC0020FEF738
:105180000FFB012014490870002509E05DF8251087
:105190002046FAF7FDFF08B16FB203E0681CC5B204
:1051A000022DF3D300BF17B1012F08D103E0012076
:1051B0000F49087007E001200D49087003E0012045
:1051C0000B49087000BF00BF0948007840B2BDE835
:1051D000FC81000018A0000858010020E405002010
:1051E000675F69656D695F6275663A2573000000E7
:1051F000510100202DE9F04105460E46002400270C
:1052000034460DE06078FFF79BF980462078FFF781
:1052100097F948EA0010C2B238467F1C2A54A41CF1
:1052200020780028EED1BDE8F08100002DE9F043A0
:10523000A9B006467048006830B16F480068FFF7B3
:1052400051FD00206C4908603EB96FF002006B49C7
:105250000968884729B0BDE8F0830120FEF7A0FA6D
:105260009620FFF7F7FB314665A0FEF7A7FA9620D8
:10527000FFF7F0FB0020FEF793FA3046FAF7B0FF95
:10528000401C84B2204601F007F905462146284615
:10529000FAF773FF224631462846FAF753FF2846AD
:1052A000FAF79EFF81464A46294620A800F0F5FEFF
:1052B00000208DF8500056E0B8F14E0F53D155A1A3
:1052C00020A800F0F2FE50B920A800F04CFE20A863
:1052D00000F049FE20A800F02CFE074643E04FA155
:1052E00020A800F0E2FE58B920A800F03CFE20A85B
:1052F00000F039FE202218A920A800F0F3FD32E0CA
:1053000048A120A800F0D1FE68BB23E0B8F14E0F01
:1053100020D146A120A800F0C8FE58B920A800F06E
:1053200022FE20A800F01FFE202210A920A800F0D5
:10533000D9FD0FE041A120A800F0B7FE50B920A888
:1053400000F011FE20A800F00EFE4022694620A8C1
:1053500000F0C8FD20A800F006FEB0F1000802D061
:1053600023980128D2DC20A800F0FDFDB0F1000850
:10537000A2D115B12846FFF7B5FCC7B10120FEF751
:105380000FFA9620FFF766FB18A92FA0FEF716FA72
:105390009620FFF75FFB0020FEF702FA174800682F
:1053A00020B16FF0020015490968884752E710A93B
:1053B0002C48FFF71FFF0120FEF7F2F99620FFF7B8
:1053C00049FB694628A0FEF7F9F99620FFF742FB52
:1053D0000020FEF7E5F969462DA003F02DFA10A98B
:1053E00030A003F029FA0548006818B101200349EC
:1053F0000968884700BF2DE7740100207001002074
:10540000726573706F6E73653D25730A28656E64EF
:10541000290A0000636F6465000000006D65737306
:105420006167650064617461000000006163636529
:1054300073735F746F6B656E00000000616363657A
:1054400073735F6164647200646576696365206C80
:105450006F67696E206661696C65643A2025730A1E
:105460000000000068010020646576696365206CB7
:105470006F67696E20737563636573732C20616356
:10548000636573735F61646472203A2025730A0058
:1054900070616E646F5F6163636573735F616464A1
:1054A0007200000070616E646F5F616363657373A7
:1054B0005F746F6B656E00002DE9F047C8B005465C
:1054C0009348006830B192480068FFF70BFC002059
:1054D0008F490860CDB90120FEF762F99620FFF7E9
:1054E000B9FA8CA0FEF76AF99620FFF7B3FA00200C
:1054F000FEF756F98D48006838B14FF0FF308B4900
:105500000968884748B0BDE8F0870120FEF748F9F0
:105510009620FFF79FFA294685A0FEF74FF99620BF
:10552000FFF798FA0020FEF73BF92846FAF758FEF5
:10553000401C84B2204600F0AFFF064621463046AC
:10554000FAF71BFE224629463046FAF7FBFD2846AD
:10555000FAF746FE8246524629463FA800F09DFDD6
:1055600067E0B8F14E0F64D176A13FA800F09DFD31
:1055700050B93FA800F0F7FC3FA800F0F4FC3FA8AA
:1055800000F0D7FCC7B254E070A13FA800F08DFD39
:1055900058B93FA800F0E7FC3FA800F0E4FC202247
:1055A00037A93FA800F09EFC43E06AA13FA800F0A5
:1055B0007CFD00283DD133E0B8F14E0F30D167A11A
:1055C0003FA800F072FD50B93FA800F0CCFC3FA806
:1055D00000F0C9FC3FA800F0B9FC814620E062A1C0
:1055E0003FA800F062FD58B93FA800F0BCFC3FA8FE
:1055F00000F0B9FC60221FA93FA800F073FC0FE087
:105600005DA13FA800F051FD50B93FA800F0ABFCF0
:105610003FA800F0A8FC602207A93FA800F062FCA8
:105620003FA800F0A0FCB0F1000802D04298012889
:10563000C2DC3FA800F097FCB0F1000891D116B190
:105640003046FFF74FFBC7B10120FEF7A9F89620BF
:10565000FFF700FA37A94BA0FEF7B0F89620FFF746
:10566000F9F90020FEF79CF83048006828B14FF0A7
:10567000FF302E490968884744E70120FEF790F87B
:105680009620FFF7E7F907AB1FAA494644A0FEF7AB
:1056900095F89620FFF7DEF90020FEF781F84A46DC
:1056A0004DA101A8FEF79AF80120FEF779F896209F
:1056B000FFF7D0F949A0FEF781F89620FFF7CAF965
:1056C0000020FEF76DF801A94DA003F0B5F81FA961
:1056D0004FA003F0B1F807A952A003F0ADF80120E4
:1056E000FEF75EF89620FFF7B5F953A0FEF766F8CF
:1056F0009620FFF7AFF90020FEF752F80B4800683C
:1057000018B1002009490968884700BFFAE600007F
:105710007C01002068747470207265717565737403
:10572000206661696C65640A000000007801002051
:10573000726573706F6E73653D25730A28656E64BC
:10574000290A0000636F6465000000006D657373D3
:1057500061676500646174610000000064657669DA
:1057600063655F69640000006465766963655F7303
:1057700065637265740000006465766963655F6BDC
:105780006579000064657669636520726567697391
:10579000746572206661696C65643A2025730A003D
:1057A00064657669636520726567697374657220E4
:1057B000737563636573732C2069643A2025642CC8
:1057C00020736563726574203A2025732C206B6505
:1057D00079203A2025730A002564000073617669F8
:1057E0006E672064657669636520696E666F2074F4
:1057F0006F2073746F726167652E2E2E0A00000091
:1058000070616E646F5F6465766963655F6964008B
:1058100070616E646F5F6465766963655F7365630D
:105820007265740070616E646F5F6465766963654C
:105830005F6B657900000000646F6E652E2E2E0A86
:10584000000000002DE9FF5F0F46944BD3E90020D4
:10585000D3E9021301AC0BC400924FF0FF390026CC
:105860003C4600E0641C20780D28FBD020780A28F4
:10587000F8D000260AE05DF826102046FAF788FCEA
:1058800010B14FFA86F903E0701CC6B2042EF2D3B1
:1058900000BFB9F1000F09D0B9F1010F2BD0B9F158
:1058A000020F6AD0B9F1030F7ED16AE07C48FFF79E
:1058B0006CF90546F5B10120FDF772FF9620FFF760
:1058C000C9F878A06968FDF779FF9620FFF7C2F85C
:1058D0000020FDF765FF29886868FDF73FFF6868CD
:1058E00020B16868FFF7FEF9002068602846FFF7DE
:1058F000F9F90025CDE070A12046FAF749FC0446ED
:1059000010342046FAF7A6FC05460120FDF748FFB3
:105910009620FFF79FF829466CA0FDF74FFF9620D1
:10592000FFF798F80020FDF73BFF42F21070854228
:105930000FDD6C48006818B100206A490968884783
:105940000020694908700846007840B204B0BDE8FC
:10595000F09F66A12046FAF71BFC0446A41C64498C
:10596000644A128888182A462146FAF7EBFB6148F8
:10597000008828445F4908808BE001205A4908705C
:1059800087E04FF000080FF2701A0120FDF708FFC2
:105990009620FFF75FF856495AA0FDF70FFF9620B3
:1059A000FFF758F8002000E072E0FDF7F9FE5146DD
:1059B0004F48FAF7EDFB0446ECB90120FDF7F0FE85
:1059C0009620FFF747F8214652A0FDF7F7FE9620F4
:1059D000FFF740F80020FDF7E3FE4248006818B1E9
:1059E000002040490968884700203F490870084660
:1059F000007840B2AAE75046FAF7F2FB00EB040B3E
:105A00005846FAF727FC0546C82D1DD00120FDF7A2
:105A1000C7FE9620FFF71EF8294644A0FDF7CEFEEC
:105A20009620FFF717F80020FDF7BAFE2D48006812
:105A300018B100202B490968884700202A490870BE
:105A40000846007840B281E741A12046FAF7A0FB62
:105A500000F104080120FDF7A3FE9620FEF7FAFFEF
:105A600041463DA0FDF7AAFE9620FEF7F3FF002079
:105A7000FDF796FE00201F49088001201A49087092
:105A80001848006818B1404616490968884700E080
:105A900000BF00BF1448007840B257E780A000085C
:105AA000DC09002073656E64696E6720446174616F
:105AB0003A25730D0A0000002B43485454504143CB
:105AC000543A20444154412C000000007265737028
:105AD0006F6E73652073697A65206973203A256457
:105AE000210A000048000020510100200D0A00009A
:105AF000F40500205C010020485454502F312E3111
:105B00002000000068747470207265636976653ADD
:105B100025730A00496E76616C696420766572733C
:105B2000696F6E20696E2025730A000072657370BC
:105B30006F6E736520636F6465206572726F72208B
:105B400069732025642C206E6F7420323030000081
:105B50000D0A0D0A000000006765742068747470F7
:105B600020726573706F6E73653A257300000000D4
:105B70002DE9F04104460D4616461F460D48006AC1
:105B8000401C0C490862086A02F020FBA060342027
:105B9000207046206070287802F00CFBE0803846C8
:105BA00002F008FBA080304602F004FB6080002079
:105BB000BDE8F0810011002010B596B0342109A88D
:105BC000FAF7DBFA15A002F02BFE0446FAF74FFBBA
:105BD000C117CDE90901154903C9CDE91201012019
:105BE000FDF7DEFD9620FEF735FF11A0FDF7E6FD7F
:105BF0009620FEF72FFF0020FDF7D2FD082112A806
:105C000003F0C4FD24220DA96846FAF79BFA09A8FF
:105C10000FC803F025FA16B010BD000070616E6465
:105C20006F5F6465766963655F6964006801002081
:105C3000746F6B656E3A0A000146032088807047D6
:105C40002DE9F04104460D46E88802F0B3FA2070D1
:105C500003F04AFC064602F0DAFAC4F80100C4F880
:105C600005101022034904F10900FAF76BFA00202D
:105C7000BDE8F0812411002010B503A105A0FEF7B6
:105C800053F80648007810BD41542B4353510D0A78
:105C90000000000041542B43535100004C000020F1
:105CA0002DE9F04385B081460F4614224F496846DE
:105CB000FAF748FA4FF0FF3800263D4600E06D1C29
:105CC00028780D28FBD028780A28F8D000260AE08A
:105CD0005DF826102846FAF75BFA10B14FFA86F8FD
:105CE00003E0701CC6B2052EF2D300BFB8F1050F59
:105CF00073D2DFE808F00326335864003C4800689C
:105D000060B13B480068006840B1394909680868DB
:105D1000FEF7E8FF0020364909680860344800684B
:105D2000FEF7E0FF00203249086001203149087089
:105D30003148006820B1002108462F4A1268904778
:105D40004CE02D48006828B14FF0FF3100202A4A6E
:105D5000126890470120274908703FE02748FEF766
:105D600014FF04460120FDF71BFD9620FEF772FE8E
:105D7000214623A0FDF722FD9620FEF76BFE0020B2
:105D8000FDF70EFD74B121886068FDF7E7FC6068DF
:105D900020B16068FEF7A6FF002060602046FEF795
:105DA000A1FF00241AE0012012490870124800687F
:105DB00020B100210846104A126890470EE00E48B4
:105DC000006828B14FF0FF3100200B4A126890475D
:105DD00001200849087001E0FFE700BF00BF054847
:105DE000007840B205B0BDE8F083000048A000088C
:105DF00034000020510100203C000020DC0900207C
:105E000073656E64696E672E2E2E2E2E2C25702CD7
:105E10000A00000008B507480068401C30B901209E
:105E200000909DF800000349086000BF0148006829
:105E300008BD00009001002010B504460E2C17D2BA
:105E4000DFE804F0160708090A0B0C0D0E0F1013FB
:105E5000141100BF00BF00BF00BF00BF00BF00BFE4
:105E600000BF00BF00BF002010BD00BF0120FBE746
:105E70000120FDF795FC9620FEF7ECFD05A0FDF74F
:105E80009DFC9620FEF7E6FD0020FDF789FCFF2033
:105E9000EAE70000556E6B6E6F77206461746120D5
:105EA000747970652E0A000010B501460A48006832
:105EB00080B10A4800680A4A126890420ADA074824
:105EC00003680068401C054C206003480068C1540A
:105ED000084610BD0020FCE7840100208C01002052
:105EE0008801002030B503460C46187E08B9002012
:105EF00030BD5869904201DB501E00E058690246EF
:105F0000002105E01D690D441868405D6054491C7E
:105F10009142F7DB00206054187EE9E70146C8682B
:105F200008B900207047C868401E01F11A02105CD1
:105F3000F8E710B50446207E302801D0002010BDBF
:105F4000226921688818FAF785F9F8E710B5044640
:105F5000207E302801D0002010BD226921688818D9
:105F6000FAF785F9F8E770B50546284603F0B2FC64
:105F7000D5E90001465C2846FFF7D0FFC4B2686847
:105F8000401C68605B2E64D006DC222E4AD02C2E8A
:105F900038D03A2E6FD12FE05D2E21D07B2E02D04B
:105FA0007D2E68D105E03146284603F0CDFA304613
:105FB00070BD3A2C08D1287E30B1284603F097FAFC
:105FC0002846FFF7ABFFC4B27B2C03D1284603F071
:105FD0008EFA03E0012068760020E9E73046E7E723
:105FE0005B2C03D1284603F082FA03E00320687695
:105FF0000020DDE73046DBE73146284603F0A4FA0F
:106000003046D5E73A2C05D1287E18B1284603F052
:106010006EFA05E05B2C03D0012068760020C7E70C
:106020003046C5E77B2C03D05B2C01D03A2C0AD13B
:106030007B2C01D14E2000E0304606460146284622
:10604000FEF724F803E0052068760020B0E730462C
:10605000AEE77B2C03D05B2C01D03A2C04D1314627
:10606000284603F071FA03E00220687600209FE7DB
:1060700030469DE7FFE73A2C01D05B2C09D1392E41
:1060800007DC302E05DB30212846FDF7FFFF3020EE
:106090008EE700BF00BF00208AE701608260002316
:1060A0004360C36043768376704770B504460D46FF
:1060B000207E10B94FF0FF3070BD23692068C118F1
:1060C00028466269FAF7B7F8F6E700002DE9F041D3
:1060D000044694F8400054F820502878492857D0B6
:1060E00004DC22284FD043287ED156E05B2802D022
:1060F0007B2879D100BF2F4694F8401004F1280086
:1061000030F811602EB92878E16B88470A20E16BDE
:1061100088477878B04207DC0A20E16B88472A7804
:10612000901CE16B884761E0002E05DD2C20E16BBF
:1061300088470A20E16B884728787B280ED1786849
:1061400050F83610204600F09BF83A20E16B884763
:10615000786800EBC600D0F8048002E0786850F858
:10616000268014F8400F401C2070002114F84029AC
:1061700004F1280020F8121094F8400044F8208020
:106180000120BDE8F0812046696800F079F82DE033
:106190002046696800F04DF828E02F4694F840103A
:1061A00004F1280030F8110008B900206064786814
:1061B00020B91CA1204600F063F814E0204679685D
:1061C000884780B194F8401004F1280030F811009D
:1061D000401C81B294F8402004F1280020F81210ED
:1061E0000120CEE700E001E00020CAE700BF94F8FC
:1061F0004000002813DD14F8400F401E207014F8F2
:10620000401904F1280030F81100401C81B294F8C4
:10621000402004F1280020F812100120B1E70020EE
:10622000AFE7000000000000002180F84010018569
:106230007047FEB506460C46002C03DA2D20F16BA4
:1062400088476442092500BF0A2094FBF0F100FB57
:1062500011403030C2B228466D1E0DF800200A20D1
:1062600094FBF0F4002C01DD002DEDDA03E01DF8C5
:106270000500F16B8847681C05460A28F7D3FEBD68
:1062800070B505460C462220E96B88476CB109E0E1
:106290002078222802D15C20E96B884714F8010B92
:1062A000E96B884720780028F2D12220E96B8847E3
:1062B00070BD000038B50120FDF772FA9620FEF798
:1062C000C9FB25A0FDF77AFA9620FEF7C3FB002054
:1062D000FDF766FA012269460B20FAF708F901205A
:1062E000FDF75EFA9620FEF7B5FB9DF8001023A09F
:1062F000FDF764FA9620FEF7ADFB0020FDF750FA9B
:10630000002414E0842000F0C7F8054604EB441193
:106310000C2202EB810188B284222946FAF7E7F8C1
:1063200021480068286020480560601CC4B29DF8C0
:1063300000008442E6DB0120FDF732FA9620FEF7EA
:1063400089FB1AA0FDF73AFA9620FEF783FB00209E
:10635000FDF726FA38BD00006C6F6164696E672036
:10636000636F6E66696720646174612066726F6D29
:1063700020666C6173682E2E2E0A000072656164BF
:10638000696E6720636F6E6669672066726F6D2045
:10639000666C6173682C206B657920636F756E7411
:1063A0003A25642E2E2E0A00A8010020646F6E6527
:1063B0002E2E2E0A0000000088B0FAF73FFD4FF4A1
:1063C000E010FCF76EFD4820FEF72EFB4FF4E130A5
:1063D00003F0D0FC4FF4E13003F006FDFBF72EFF95
:1063E000FAF781F808E03220FEF728FB0120254962
:1063F00008603220FEF722FBFAF75EF80028F2D19F
:106400001F226946FAF773F801201E49086037E039
:10641000FEF7E6FCB0F1FF3F02D100F0DFFB21E028
:10642000FEF7DEFC012802D100F052FB1AE0FEF775
:10643000D7FC032816D1042003F0A2F90120FDF7B0
:10644000AFF99620FEF706FB0FA0FDF7B7F99620EF
:10645000FEF700FB0020FDF7A3F9002009490860C2
:1064600002F07EFC08E0206810B1D4E900108847F3
:1064700014B12046FEF733FB03F046F8041EF2D1B8
:10648000C6E7000080012242496E697420476574A6
:106490007761790D0A000000F0B50B30154D20F042
:1064A00007010024144A0FE003688B420BD38B4290
:1064B00005D95E1A43184768C3E9006700E04368DE
:1064C000136002C004E0021D10680028ECD12046D1
:1064D000002802D1286808B10020F0BD064A07480C
:1064E0001060074A121A22F00702C0E900240120B6
:1064F0002860D7E7B8010020B40100202C13002049
:1065000028330020F8B50646002000903446A088C5
:1065100003281DDA0120FDF743F99620FEF79AFAC9
:1065200040A0FDF74BF99620FEF794FA0020FDF706
:1065300037F954B1206820B12068FEF7D3FB002062
:1065400020602046FEF7CEFB00244FF0FF30F8BD60
:106550003E480078B0B93EA12068F9F719FE88B12D
:106560000120FDF71DF99620FEF774FA39A0FDF71A
:1065700025F99620FEF76EFA0020FDF711F90120AB
:106580003249087031480078022803D02F4800783B
:10659000042839D100253748006810B300BF1DE03A
:1065A000354850F8351033480068F9F720FEA0B997
:1065B000314800EBC50021684268684690472F4982
:1065C000087008460078012806D12A480068FEF7BE
:1065D00089FB00202749086002E06D1C182DDFD3DD
:1065E00011E02046FEF740F9012809D1244800684F
:1065F00048B104220020224B21681B68984702E022
:10660000204603F02DFC00BF54B1206820B1206863
:10661000FEF768FB002020602046FEF763FB0024A5
:10662000002094E76D6F64756C6520726573706F00
:106630006E7365206E6F7420656E6F756768206C71
:10664000656E677468210D0A00000000500100208B
:106650004F4B0000746865202261742220636D64D2
:1066600020726573706F6E736520224F4B220D0A86
:1066700000000000540100205000002051010020C3
:10668000400000202DE9F74FDAB004468A469249CF
:106690005C98086040214AA8F9F76FFD40213AA8AC
:1066A000F9F76BFD4FF0500807228CA12046F9F74F
:1066B000C2FD08B9012000E000203990082289A11C
:1066C0002046F9F7B8FD08B9012000E00020389015
:1066D000399808B1E41D17E0389818B1083440F231
:1066E000BB1811E00120FDF75BF89620FEF7B2F928
:1066F0007FA0FDF763F89620FEF7ACF90020FDF7C8
:106700004FF85DB0BDE8F08F2F212046F9F75EFD10
:10671000054625B900212046F9F758FD05463A21DE
:106720002046F9F753FD0646AE4200D900262EB9A1
:106730002A1B21464AA8F9F705FD10E0701CF9F75D
:1067400089FD8046B8F1000F00D1DAE7321B2146FF
:106750004AA8F9F7F7FC0020311B4AAA5054002040
:10676000291B4AAA50542046F9F73AFD83464AA805
:10677000F9F736FDABEB00000246294602903AA835
:10678000F9F7E0FC0120FDF70BF89620FEF762F91F
:106790004AA95FA0FDF712F89620FEF75BF90020EA
:1067A000FCF7FEFF0120FCF7FBFF9620FEF752F9F5
:1067B0003AA95BA0FDF702F89620FEF74BF90020FE
:1067C000FCF7EEFF0120FCF7EBFF9620FEF742F905
:1067D000414657A0FCF7F2FF9620FEF73BF9002058
:1067E000FCF7DEFF56A15AA0FDF79EFA5BA15FA061
:1067F000FDF79AFA402128A8F9F7BFFC4AAB01221D
:106800005DA128A8CDF80080FCF7E8FF0120FCF787
:10681000C7FF9620FEF71EF928A95EA0FCF7CEFF61
:106820009620FEF717F90020FCF7BAFF28A95FA011
:10683000FDF77AFA802108A8F9F79FFC142103A834
:10684000F9F79BFC5046F9F7CBFC83465A465AA110
:1068500008A8FCF7C3FF0820FFF71EFE07464FF409
:106860000070FFF719FE786008A8CDE9010ACDF89D
:1068700000804AAB3AAA5D497868FCF7AFFF8146D1
:10688000A7F800900120FCF78BFF9620FEF7E2F8B6
:106890004A4657A07968FCF791FF9620FEF7DAF890
:1068A0000020FCF77DFF4B46012257A103A8FCF70F
:1068B00095FF03A959A0FDF737FA39465A48FEF764
:1068C0006CF95AA15DA0FDF72FFA5FA162A0FDF758
:1068D0002BFA00BF15E700004800002068747470B0
:1068E0003A2F2F0068747470733A2F2F0000000045
:1068F00075726C206973206E6F7420687474703ABE
:106900002F2F206F722068747470733A2F2F00003D
:10691000686F73745F6E616D653A25730A000000DD
:10692000687474705F706174683A25730A000000BF
:10693000687474705F706F72743A25640A000000A6
:1069400041542B4343485345543D310D0A00000048
:1069500041542B43434853455400000041542B43BA
:10696000434853544152540D0A00000041542B43F4
:10697000434853544152540041542B4343484F50D1
:10698000454E3D25642C222573222C25642C310D87
:106990000A000000726561647920746F2068747465
:1069A0007020706F73743A257300000041542B43BC
:1069B00043484F50454E0000436F6E74656E742D12
:1069C000547970653A6170706C69636174696F6E57
:1069D0002F6A736F6E0D0A436F6E74656E742D4C63
:1069E000656E6774683A2025640D0A0098A4000853
:1069F0006874747020706F73743A25732C206C6502
:106A00006E3A25640000000041542B43434853452F
:106A10004E443D25642C25640D0A000041542B434F
:106A2000434853454E440000DC09002041542B43A9
:106A30004348434C4F53453D310D0A0041542B43CD
:106A40004348434C4F53450041542B434348535410
:106A50004F500D0A0000000041542B43434853544B
:106A60004F500000F0B58DB007460E461446082082
:106A7000FFF712FD05462C802046FFF70DFD6860EC
:106A8000224631466868F9F75DFB2346012207A1DB
:106A900001A8FCF7A3FE01A909A0FDF745F92946C5
:106AA0000A48FEF77AF80DB0F0BD000041542B43C0
:106AB000495053454E443D25642C25640D0A000081
:106AC00041542B43495053454E440000DC090020FB
:106AD00010B514A0FCF750FE1748F9F7D8FD17A120
:106AE00018A0FDF721F918A11AA0FDF71DF91BA1A7
:106AF0001DA0FDF719F91EA120A0FDF715F921A190
:106B000024A0FDF711F926A129A0FDF70DF92BA16D
:106B10002EA0FDF709F902202F49087008460078D9
:106B200010BD00006D6F64756C655F696E697421DE
:106B300021210D0A00000000DC09002041544530ED
:106B40000D0A00004154450041542B4350494E3F2B
:106B50000D0A000041542B4350494E0041542B4331
:106B600053510D0A0000000041542B4353510000C3
:106B700041542B4347534E0D0A00000041542B4310
:106B800047534E0041542B4349504D4F44453D30EF
:106B90000D0A000041542B4349504D4F444500001D
:106BA00041542B4E4554434C4F53450D0A000000B1
:106BB00041542B4E4554434C4F53450041542B4EAA
:106BC00045544F50454E0D0A0000000041542B4ED5
:106BD00045544F50454E00005001002010B5002094
:106BE00006490870064A01214FF47A7003F02CF828
:106BF00003F068F80148007810BD00005001002043
:106C0000793E00082DE9F74398B0814614460EA15D
:106C100011A0FDF789F89DF864509DF865609DF816
:106C200066709DF867802B4601220EA104A88DE8AE
:106C3000C0010394FCF7D2FD04A914A0FDF774F879
:106C40001BB0BDE8F083000041542B434950434C36
:106C50004F53453D310D0A0041542B434950434C9D
:106C60004F53450041542B4349504F50454E3D250D
:106C7000642C22544350222C2225642E25642E2578
:106C8000642E2564222C25640D0A000041542B43F8
:106C900049504F50454E000070B504460120FCF7A6
:106CA0007FFD9620FDF7D6FE07A0FCF787FD962016
:106CB000FDF7D0FE0020FCF773FD254607490120B3
:106CC00001F042FC70BD00004D5154543A20436F16
:106CD0006E6E65637465640D0A00000051910008D2
:106CE0002DE9F84F8A4617469946DDF8288001209D
:106CF000FCF756FD9620FDF7ADFE94A0FCF75EFD77
:106D00009620FDF7A7FE0020FCF74AFD0120FCF7C6
:106D100047FD9620FDF79EFE394690A0FCF74EFDFC
:106D20009620FDF797FE0020FCF73AFD0120FCF7C6
:106D300037FD9620FDF78EFE41468EA0FCF73EFD06
:106D40009620FDF787FE0020FCF72AFD002000902A
:106D5000BAF1000F02D0B9F1000F10D10120FCF7F9
:106D60001FFD9620FDF776FE88A0FCF727FD9620F4
:106D7000FDF770FE0020FCF713FDBDE8F88F781CCE
:106D8000FFF78AFB0646791C3046F9F7F6F93A46D2
:106D900051463046F9F7D6F90020F0550120FCF7AE
:106DA000FFFC9620FDF756FE31467EA0FCF706FD5F
:106DB0009620FDF74FFE0020FCF7F2FC4FF0000B91
:106DC0003078632808D064280CD0652807D0732851
:106DD0000BD14FF0030B09E04FF0010B06E04FF031
:106DE000020B03E04FF0030B00E0C6E700BF1EB14B
:106DF0003046FDF777FF00260820FFF74DFB0446DD
:106E00007CB90120FCF7CCFC9620FDF723FE6AA09C
:106E1000FCF7D4FC9620FDF71DFE0020FCF7C0FC1B
:106E2000ABE7A4F800804046FFF736FB606060687F
:106E300078B90120FCF7B4FC9620FDF70BFE5EA0AC
:106E4000FCF7BCFC9620FDF705FE0020FCF7A8FC33
:106E500093E7606842464946F9F774F9002060807C
:106E60006946204602F0D2F80120FCF799FC9620F2
:106E7000FDF7F0FD54A0FCF7A1FC9620FDF7EAFD1C
:106E80000020FCF78DFC2188606802F07FFC5946E9
:106E9000204601F0F3FF78B10120FCF781FC962039
:106EA000FDF7D8FD53A0FCF789FC9620FDF7D2FD35
:106EB0000020FCF775FC60E70620FFF7EDFA0546B9
:106EC00020886188401A28802888FFF7E5FAC5F8ED
:106ED00002006368B4F802C003EB0C012A88D5F8FD
:106EE0000200F9F72FF9204601F05FFBBDF8000022
:106EF000012805D0BDF800004FF6FF71884217D178
:106F00000120FCF74DFC9620FDF7A4FDBDF8001014
:106F100040A0FCF753FC9620FDF79CFD0020FCF7F9
:106F20003FFC2A88D5F802100120FDF7F3FA08E0AB
:106F3000BDF8000028B92A88D5F802100020FDF716
:106F4000E9FA2846FDF7AAFD00BF16E76D717474D3
:106F50005F646174615F63620A0000006D71747444
:106F600020746F706963206C656E6774683A2025C1
:106F7000640A00006D7174742064617461206C6532
:106F80006E6774683A2025640A0000006E6F206EF8
:106F90006565646564206D717474207061636B61F4
:106FA0006765210074686520746F70696320697378
:106FB0003A2025730A0000006D616C6C6F632065D8
:106FC00072726F72210A00007061636B61676520E5
:106FD00066726F6D207365727665722C20676574BA
:106FE00020726964206F66206D7174742068656119
:106FF000643A0A0074686520646174612066726F87
:107000006D207365727665722069732077726F6E7A
:1070100067210A007472616E736665722064617420
:107020006120746F20737562206465766963653AC8
:107030002025640A0000000070B504460120FCF71A
:10704000AFFB9620FDF706FD05A0FCF7B7FB9620E9
:10705000FDF700FD0020FCF7A3FB254670BD0000F6
:107060004D5154543A20446973636F6E6E65637476
:1070700065640D0A0000000010B504460120FCF70D
:107080008FFB9620FDF7E6FC08A0FCF797FB962007
:10709000FDF7E0FC0020FCF783FB0B48006820B103
:1070A0006FF0030008490968884710BD4D515454DA
:1070B0003A20636F6E6E656374696E6720657272E5
:1070C0006F720D0A00000000640100202DE9F041FC
:1070D00005460E46012E02DA0020BDE8F08100BF11
:1070E00028780009C01E09284AD2DFE800F00536DA
:1070F0003738393C3A493B00012406E0285D00F06E
:10710000800008B9641C02E0641CB442F6DB00BFD6
:10711000A01CB04201DB0020DFE72046641C285C95
:1071200007022046641C285C0743E019B04201DBDB
:107130000020D2E73C44284600F0A5F8002804DDF2
:10714000A01CB04203DB0020C7E70020C5E7601C9D
:10715000285C295D40EA0120BFE700BF00BF00BFF7
:1071600000BF00BF00BF042E08DB687800F080007D
:1071700020B9E878A97840EA0120AEE70020ACE722
:107180000020AAE72DE9F04106460D46002701241C
:107190000EE0305D00F07F00611EC1EBC101884050
:1071A0000744305D00F0800008B9641C03E0641CF3
:1071B0002888A042EDDC00BF27442988A01C81421A
:1071C00002DC0020BDE8F0812046641C305C4FEA00
:1071D00000282046641C305C40EA080804EB0800E4
:1071E0002988884202DB00202880EBE744443046AF
:1071F00000F049F8002806DD2988A01C814201DC46
:107200000020DFE7A41CA74201DA0020DAE7288883
:10721000B84202DB381B288002E02888001B288047
:107220003019CFE770B502460B46002501210EE06C
:10723000505C00F07F004E1EC6EBC606B040054411
:10724000505C00F0800008B9491C03E0491C188814
:107250008842EDDC00BF0D441E88881C864201DC9C
:10726000002070BD0846491C105C04020846491CF9
:10727000105C044308191E88B04201DD0020F0E7CD
:107280001C805018EDE701460878C0F341007047B4
:1072900030B502460B46002001210EE0545C04F09C
:1072A0007F044D1EC5EBC505AC402044545C04F082
:1072B00080040CB9491C02E0491C9942EEDB00BF76
:1072C000084430BD0146087800097047F8B5064605
:1072D0000C463046FEF7B0FCB0880A30318A88424E
:1072E00003D93046FDF74CFCF8BDB188F06845186D
:1072F000B0880A30B08000202870042068704CA04C
:107300000068C5F802000420A8710020E871A08A76
:10731000000A2872207D6872206A18B1E87940F06E
:107320000200E871206888B12068007870B1206898
:10733000F8F756FF07463A4630462168FCF776FDD7
:10734000002807DA3046FDF71BFCCDE73046FDF795
:1073500017FCC9E7E06888B3E068007870B3E068BC
:10736000F8F73EFF07463A463046E168FCF75EFD17
:10737000002803DA3046FDF703FCB5E72069F8F78B
:107380002FFF07463A4630462169FCF74FFD00289B
:1073900003DA3046FDF7F4FBA6E7E87940F0040095
:1073A000E871E06918B1E87940F02000E871E87907
:1073B000217E01F0030140EAC100E8716068A8B1D4
:1073C0006068007890B16068F8F70AFF07463A46AF
:1073D00030466168FCF72AFD002803DA3046FDF7E5
:1073E000CFFB81E7E87940F08000E871A068A8B1A0
:1073F000A068007890B1A068F8F7F2FE07463A4618
:107400003046A168FCF712FD002803DA3046FDF78C
:10741000B7FB69E7E87940F04000E87100200346D7
:107420000246012100903046FDF704FC5CE70000B5
:107430004D5154540000000000230360C1600282DB
:10744000704738B504462046FEF7F6FB0020034699
:1074500002460C2100902046FDF7ECFB38BD38B504
:1074600004462046FEF7E8FB0020034602460D21B5
:1074700000902046FDF7DEFB38BD38B504460D46CA
:107480002046FEF7D9FB29462046FCF7B1FC18B987
:107490002046FDF775FB38BD002003460246042157
:1074A00000902046FDF7C6FBF5E738B504460D46CB
:1074B0002046FEF7C1FB29462046FCF799FC18B987
:1074C0002046FDF75DFB38BD00200346024607213C
:1074D00000902046FDF7AEFBF5E72DE9F84F044696
:1074E0000D4617461E46DDE90BA9DDF8288020462B
:1074F000FEF7A2FB0DB1287820B92046FDF740FB2E
:10750000BDE8F88F2846F8F76BFE83465A462946B1
:107510002046FCF78BFC002803DA2046FDF730FB01
:10752000EEE7B8F1000F0ADD00212046FCF760FC11
:10753000A9F8000030B92046FDF722FBE0E7002063
:10754000A9F80000A0883044218A884203DD204643
:10755000FDF716FBD4E7A288E16888183246394661
:10756000F8F7F0FDA0883044A080434600220321B4
:107570002046CDF800A0FDF75DFBC1E738B5044615
:107580000D462046FEF758FB29462046FCF730FC06
:1075900018B92046FDF7F4FA38BD0020034602462C
:1075A000052100902046FDF745FBF5E738B5044678
:1075B0000D462046FEF740FB29462046FCF718FC06
:1075C00018B92046FDF7DCFA38BD00200123024639
:1075D000062100902046FDF72DFBF5E770B5044627
:1075E0000120FCF7DDF89620FDF734FA05A0FCF742
:1075F000E5F89620FDF72EFA0020FCF7D1F8254695
:1076000070BD00004D5154543A205075626C69733E
:107610006865640D0A0000002DE9FC4105460F462F
:107620002E46746A3149304600F03AFF3049304600
:1076300000F042FF2F49304600F04AFF0120FCF7DE
:10764000AFF89620FDF706FA2BA0D4E90212FCF75A
:10765000B5F89620FDF7FEF90020FCF7A1F8A08D03
:1076600082B204F13800616AFFF7E6FE04F13800E7
:10767000E169FFF72BFE6063616B0868FFF722FE8C
:107680002065626B91881068FFF720FD4C2108533C
:107690000520C4F8A800606B8088ADF80000606B1E
:1076A000006801900120FCF77BF89620FDF7D2F9E5
:1076B0004C20025B19A0216DFCF780F89620FDF7A5
:1076C000C9F90020FCF76CF8B4F8A80083B2304682
:1076D000DDE9001200F008FF002161630C2084F84E
:1076E000B0002046FBF736F8BDE8FC814177000882
:1076F000A9770008CD7E00084D5154543A20436FBD
:107700006E6E656374656420746F2062726F6B6562
:10771000722025733A25640D0A0000004D5154541F
:107720003A2053656E64696E672C20747970653AEF
:107730002025642C2069643A20253034580D0A0035
:107740002DE9F04105460F462E46746A0120FCF7EC
:1077500027F89620FDF77EF90BA0FCF72FF896206E
:10776000FDF778F90020FCF71BF8062084F8B0003C
:10777000D4F8800018B12046D4F8801088472046FD
:10778000FAF7E8FFBDE8F0815443503A20446973AA
:10779000636F6E6E65637465642063616C6C6261B7
:1077A000636B0D0A000000002DE9FE4F83460E4674
:1077B0000120FBF7F5FF9620FDF74CF93188FEA07C
:1077C000FBF7FCFF9620FDF745F90020FBF7E8FFEB
:1077D000CDF808B0DDF808B0DBF824403088B0F50B
:1077E000806F01DC308880B90120FBF7D9FF96203B
:1077F000FDF730F9F8A0FBF7E1FF9620FDF72AF935
:107800000020FBF7CDFFBDE8FE8F638ED4F820C0CB
:107810000CEB030032887168F8F794FC608E3188B5
:107820000844608600BF608E01280ED1FBF7B8FFC8
:107830009620FDF70FF9EFA0FBF7C0FF9620FDF7AC
:1078400009F90020FBF7ACFFDDE7618E206AFFF746
:107850001FFD20860120FBF7A3FF9620FDF7FAF815
:10786000218EEFA0FBF7AAFF9620FDF7F3F800208A
:10787000FBF796FF618E206A01F088FF218E608EF3
:1078800081420FDD0120FBF78BFF9620FDF7E2F828
:10789000E8A0FBF793FF9620FDF7DCF80020FBF74C
:1078A0007FFFB0E7206AFFF70DFD00F0FF09206AB7
:1078B0000178C1F3410500BF218E206AFFF706FC65
:1078C00007460120FBF76CFF9620FDF7C3F8208EDA
:1078D000CDE9007094F8B0102B464A46DA48FBF721
:1078E0006DFF9620FDF7B6F80020FBF759FF94F8DE
:1078F000B0000C2802D00F2832D132E0B9F1020FCB
:107900002ED1206D012812D00120FBF749FF9620CF
:10791000FDF7A0F8CDA0FBF751FF9620FDF79AF8F0
:107920000020FBF73DFF206800F096FD18E00120E5
:10793000FBF736FF9620FDF78DF8CAA0D4E90212B6
:10794000FBF73CFF9620FDF785F80020FBF728FFAA
:107950000F2084F8B000E06F10B12046E16F884737
:1079600021E1A9F103000B281DD2DFE800F0347BF0
:1079700092B1D01C061C1DE7FD00206D082806D121
:107980004C20005BB84202D10120FBF709FF962092
:10799000FDF760F8BAA0FBF711FF9620FDF75AF843
:1079A0000020FBF7FDFEFCE0206D0A2806D14C20EC
:1079B000005BB84202D10120FBF7F2FE9620FDF7F2
:1079C00049F8B7A0FBF7FAFE9620FDF743F8002030
:1079D000FBF7E6FEE5E0012D06D1394604F138005B
:1079E000FFF74BFD606307E0022D05D1394604F136
:1079F0003800FFF7C3FD6063012D01D0022D27D1B0
:107A00000120FBF7CDFE9620FDF724F82946ACA017
:107A1000FBF7D4FE9620FDF71DF80020FBF7C0FE13
:107A2000606B8288016804F1B400FBF7ECF8401C3D
:107A300070B90120FBF7B4FE9620FDF70BF8A8A063
:107A4000FBF7BCFE9620FDF705F80020FBF7A8FE2B
:107A5000218E206A01F09AFE228E2046216AFDF7CF
:107A60004FF89EE0206D032812D14C20005BB842F5
:107A70000ED10120FBF794FE9620FCF7EBFF9DA0B2
:107A8000FBF79CFE9620FCF7E5FF0020FBF788FE45
:107A900087E0394604F13800FFF788FD6063606BCA
:107AA0008288016804F1B400FBF7ADF8401C70B99E
:107AB0000120FBF775FE9620FCF7CCFF88A0FBF7B2
:107AC0007DFE9620FCF7C6FF0020FBF769FE68E00C
:107AD000394604F13800FFF7E8FC6063606B828888
:107AE000016804F1B400FBF78EF8401C70B9012066
:107AF000FBF756FE9620FCF7ADFF79A0FBF75EFE84
:107B00009620FCF7A7FF0020FBF74AFE49E0206D16
:107B1000032812D14C20005BB8420ED10120FBF7A4
:107B20003FFE9620FCF796FF81A0FBF747FE9620CC
:107B3000FCF790FF0020FBF733FE32E004F1380041
:107B4000FFF78DFC6063606B8288016804F1B4000C
:107B5000FBF759F8401C80B90120FBF721FE962065
:107B6000FCF778FF5EA000E008E0FBF727FE962018
:107B7000FCF770FF0020FBF713FE12E00120FBF77B
:107B80000FFE9620FCF766FF78A0FBF717FE962005
:107B9000FCF760FF0020FBF703FE0120C4F8AC00F7
:107BA00000BF00BF00BF00BF618E208E081A1FFA01
:107BB00080F8A4F83280E9E05443503A20646174BC
:107BC0006120726563656976656420256420627949
:107BD0007465730D0A00000072656365697665203F
:107BE0006C656E67746820697320696E76616C6974
:107BF000642E0A006E6F7420656E6F75676820646E
:107C000061746120666F72207265616420706163C7
:107C10006B616765206C656E6774682E0A210000D1
:107C20006D657373616765206C656E6774683A256E
:107C3000640A00006E6F7420656E6F75676820645B
:107C40006174612E0A000000B4A500084D5154541F
:107C50003A20496E76616C6964207061636B65746B
:107C60000D0A00004D5154543A20436F6E6E656307
:107C700074656420746F2025733A25640D0A000032
:107C80004D5154543A205375627363726962652092
:107C90007375636365737366756C0D0A000000008D
:107CA0004D5154543A20556E537562736372696234
:107CB00065207375636365737366756C0D0A0000E8
:107CC0004D5154543A205175657565207265737035
:107CD0006F6E736520516F533A2025640D0A0000C2
:107CE0004D5154543A2051756575652066756C6C1C
:107CF0000D0A00004D5154543A207265636569764F
:107D00006564204D5154545F4D53475F545950455D
:107D10005F50554241434B2C2066696E6973682061
:107D2000516F5331207075626C6973680D0A0000E1
:107D30004D5154543A2072656365697665204D5102
:107D400054545F4D53475F545950455F505542431B
:107D50004F4D502C2066696E69736820516F533205
:107D6000207075626C6973680D0A00007265636546
:107D7000697665206120686561727420626561744E
:107D800020726573706F6E7365210A000120FBF726
:107D900007FD9620FCF75EFE618E2AA0FBF70EFD24
:107DA0009620FCF757FE0020FBF7FAFC0120FBF7BA
:107DB000F7FC9620FCF74EFE218E2EA0FBF7FEFC72
:107DC0009620FCF747FE0020FBF7EAFC0120FBF7BA
:107DD000E7FC9620FCF73EFE30A0FBF7EFFC962078
:107DE000FCF738FE0020FBF7DBFC218E206A01F057
:107DF000CDFCB8F1000F20DD4FF0000A00BF0AE013
:107E0000608EA0EB08005044216A095C206A00F8EB
:107E10000A100AF1010AC245F2DB0120FBF7C0FC9F
:107E20009620FCF717FE21A0FBF7C8FC9620FCF774
:107E300011FE0020FBF7B4FCF5E42046FAF78AFCBB
:107E400000BFE0E4636C69656E742D3E6D717474FF
:107E50005F73746174652E6D6573736167655F6CC4
:107E6000656E6774685F72656164203D2025640AF1
:107E700000000000636C69656E742D3E6D71747452
:107E80005F73746174652E6D6573736167655F6C94
:107E9000656E677468203D2025640A00746865205B
:107EA0007061636B6167652069730A0047657420C0
:107EB000616E6F74686572207075626C6973686555
:107EC00064206D6573736167650D0A002DE9F041EB
:107ED00005460E462F467C6A06BB0120FBF760FC78
:107EE0009620FCF7B7FD1BA0FBF768FC9620FCF77B
:107EF000B1FD0020FBF754FC0020C4F8A80094F862
:107F0000B0000F2821D1206D03281ED1D4F88400A1
:107F1000D8B12046D4F88410884716E0701CA0B968
:107F20000120FBF73DFC9620FCF794FD0DA0FBF72C
:107F300045FC9620FCF78EFD0020FBF731FC00206D
:107F4000C4F8A800062084F8B0002046FAF702FC26
:107F5000BDE8F0815443503A2053656E74204F4B76
:107F60000D0A00005443503A2073656E7420666118
:107F7000696C6564210000007CB505462C46012033
:107F8000FBF70EFC9620FCF765FD94F8B0206349E2
:107F900063A0FBF713FC9620FCF75CFD0020FBF7C9
:107FA000FFFB94F8B0000F2862D154F89C0F401CDE
:107FB000206054F89C19E0694069814257D9D4F88F
:107FC000AC0010B9062084F8B0000120FBF7E8FBF4
:107FD0009620FCF73FFD54A0D4E90212FBF7EEFB1C
:107FE0009620FCF737FD0020FBF7DAFB04F13800A0
:107FF000FFF727FA60630C212165616B0868FFF7C2
:1080000061F92065626B91881068FFF75FF84C2179
:1080100008530520C4F8A800606B8088ADF8000004
:10802000606B006801900120FBF7BAFB9620FCF71B
:1080300011FD4C20025B47A0216DFBF7BFFB962092
:10804000FCF708FD0020FBF7ABFBB4F8A8108BB2DF
:108050002068DDE9001200F047FA0021616300208A
:10806000C4F89C00C4F8AC002046FAF773FB4CE05F
:1080700094F8B000062822D10120FBF791FB96204E
:10808000FCF7E8FC54F8A02F24493BA0FBF796FB33
:108090009620FCF7DFFC0020FBF782FB2068401CE9
:1080A000206054F8A00905282FD90020C4F8A000AA
:1080B000072084F8B0002046FAF74CFB25E094F83E
:1080C000B000082821D10120FBF76AFB9620FCF7BD
:1080D000C1FC54F8A42F11492FA0FBF76FFB962089
:1080E000FCF7B8FC0020FBF75BFB2068401C20601D
:1080F00054F8A409142808D9092084F8B0000020F5
:10810000C4F8A4002046FAF725FBD4F8A80020B153
:10811000D4F8A800401EC4F8A8007CBD6DA10008DA
:1081200025732C2025640A000D0A4D5154543A2021
:1081300053656E64206B656570616C69766520704F
:1081400061636B657420746F2025733A2564210D7B
:108150000A0000004D5154543A2053656E64696E14
:10816000672C20747970653A2025642C2069643A64
:1081700020253034580D0A0025732C20636C696566
:108180006E742D3E7265636F6E6E656374546963C1
:108190006B3A25640A00000025732C20636C696526
:1081A0006E742D3E636F6E6E6563745469636B3AD3
:1081B00025640A0000B50246FDF72CFE20B1100A26
:1081C000D1B240EA012000BD1046FCE700B50246EE
:1081D000FDF720FE58B1100E02F47F0140EA112095
:1081E00002F47F4140EA012040EA026000BD1046EF
:1081F000FCE718B50446FDF70DFE30B10094009879
:10820000FFF7E4FF0090009818BD2046FCE72DE939
:10821000F04106460F46FF240025FDF7FBFD002830
:108220003DD007EA0460020E002107EA044042EA5A
:1082300010200943002307EA042C43EA0C220B46D2
:1082400040EA020143EA1C6004EA07034FEA036CB8
:1082500041EA0C0240EA1323290641EA142106EA06
:10826000046C3940080240EA1C6042EA0C210343D6
:10827000280440EA144006EA04423840000640EA76
:10828000122C41EA026043EA0C0106EA042241EAA8
:10829000022106EA040241EA0261BDE8F0813046AB
:1082A0003946FAE77CB504460D46FDF7B3FD58B1F3
:1082B000CDE90045DDE900211046FFF7A8FFCDE933
:1082C0000001DDE900017CBD20462946FBE70000F6
:1082D0002DE9FF4180460E461F4B0FCB8DE80F0066
:1082E0004FF0FF370025344600E0641C20780D284D
:1082F000FBD020780A28F8D0002509E05DF8251089
:108300002046F7F745FF08B16FB203E0681CC5B21D
:10831000042DF3D300BF37B1012F08D0022F0AD0AC
:10832000032F10D10BE001200C4908700CE0012054
:108330000A49087008E001200849087004E001209B
:108340000649087000E000BF00BF0448007840B252
:1083500004B0BDE8F08100002CA00008510100200D
:1083600010B50024FDF788FC04460C2C01DD01202B
:1083700010BD0020FCE770B504460D461646324697
:1083800029462046FEF77EF970BD00002DE9FE4328
:1083900080460E461D4A07CA8DE807004FF0FF379A
:1083A0000025344600E0641C20780D28FBD020789E
:1083B0000A28F8D0002509E05DF825102046F7F7D7
:1083C000E7FE08B16FB203E0681CC5B2032DF3D31A
:1083D00000BF27B1012F03D0022F0FD107E00EE01D
:1083E00001200B49087003200A49087007E00120AA
:1083F0000749087003200749087000E000BF00BF6C
:108400000348007840B2BDE8FE83000020A00008C9
:1084100051010020500100202DE9F041044688461A
:1084200066682789002500BF09E00A4850F8250042
:1084300020B96582074840F8254002E06D1C0A2DEE
:10844000F3DB00BF608A3A463146FEF7DBFBBDE84E
:10845000F0810000801200200146002000BF0CE0E7
:108460004A8A084B53F820305B8A9A4204D1002292
:10847000044B43F8202002E0401C0A28F0DB00BF38
:10848000704700008012002070B504460D466561FB
:10849000608A024901F06AF870BD0000B9990008CD
:1084A00070B504460D4625620249002001F064F8CB
:1084B00070BD00005D9A000870B504460D46A561C8
:1084C0000249002001F05EF870BD0000E59A000846
:1084D00070B504460D46E5610249002001F058F8E8
:1084E00070BD0000499B00087FB504461D46012071
:1084F000FBF756F99620FCF7ADFA0B490BA0FBF7FA
:108500005DF99620FCF7A6FA0020FBF749F9BDF8C3
:108510000410029801F03AF9BDF8042000200299F5
:10852000FEF7A0FA7FBD0000C5A1000825732C74DA
:1085300063702073656E640A0000000010B50820A7
:10854000FDF7AAFF10BD000000EB4002024B03EB59
:108550008202916070470000B00F002000EB4002E3
:10856000024B03EB8202516070470000B00F002005
:1085700070B505460E460820FDF78EFF04460CB97F
:10858000002070BD258066802088FDF785FF606033
:10859000606820B92046FCF7A5FB0020F1E72188A0
:1085A0006068F7F7EAFD2046EBE710B5044604B92A
:1085B00010BD606810B16068FCF794FB2046FCF7C2
:1085C00091FB00BFF4E700002DE9F04397B00446AB
:1085D0000120FBF7E5F89620FCF73CFA53A0FBF7E7
:1085E000EDF89620FCF736FA0020FBF7D9F80120C9
:1085F000FBF7D6F89620FCF72DFA54A0FBF7DEF82F
:108600009620FCF727FA0020FBF7CAF80CB1534874
:10861000046053A000F004F90546B5B90120FBF74A
:10862000BFF89620FCF716FA52A0FBF7C7F8962081
:10863000FCF710FA0020FBF7B3F86FF0030047498E
:108640000968884717B0BDE8F08316AA12A9284622
:10865000FBF7ACFFA0B10120FBF7A2F89620FCF7D6
:10866000F9F94DA0FBF7AAF89620FCF7F3F90020E2
:10867000FBF796F86FF00300384909688847E1E78F
:108680004DA000F0CDF880464046F7F7F0FD81465A
:108690004A464DA14D48FBF7A1F8FDF78DFA01239D
:1086A00012A94B48169AF9F747FF4AA000F0B8F80C
:1086B00007463846F7F794FD461C3246394602A86D
:1086C000F7F740FD01201E2102AB47A2CDE90010C3
:1086D0003E493F48F9F7A0FE0120FBF761F89620DC
:1086E000FCF7B8F9394941A0FBF768F89620FCF788
:1086F000B1F90020FBF754F844493548F9F75DFF1C
:1087000043493348F9F75EFF42493148F9F75DFFC5
:1087100041492F48F9F753FF40492D48F9F74AFFDF
:108720002B48F9F7BFFD00BF8CE7000050414E44D5
:108730004F3A20626567696E2061636365737320D9
:10874000636C6F75642E2E2E0A0000006265666FE2
:108750007265206163636573733A0A0064010020E7
:1087600070616E646F5F6163636573735F6164649E
:10877000720000006E6F2061636365737320736520
:1087800072766572206164647265737320666F75BA
:108790006E642E2E2E0A000077726F6E6720616362
:1087A00063657373207365727665722061646472A9
:1087B0006573732E2E2E0A0070616E646F5F6465A0
:1087C000766963655F69640025780000E010002029
:1087D0001010002070616E646F5F61636365737376
:1087E0005F746F6B656E000000000000616363657D
:1087F0007373207374725F6465766963655F69641F
:108800005F6865783A25730A00000000996C0008DB
:1088100039700008DD750008E16C00087970000807
:1088200070B505462846FCF7BFF9044614B104F1BB
:10883000240070BD0020FCE72DE9F04106460F46FC
:108840003046FCF7B1F90546C5B16022394605F15D
:108850002400F7F7AFFC0120FAF7A2FF9620FCF7FF
:10886000F9F805F1240231461AA0FAF7A7FF96207D
:10887000FCF7F0F80020FAF793FF26E08420FDF7DC
:108880000BFE044620223146201DF7F793FC6022A0
:10889000394604F12400F7F78DFC15480068206084
:1088A000134804600120FAF77BFF9620FCF7D2F80A
:1088B00004F1240231460FA0FAF780FF9620FCF75E
:1088C000C9F80020FAF76CFF00BF00F067FE012036
:1088D000BDE8F0816B657920257320757064617443
:1088E00065642C76616C75653A25730A000000009A
:1088F000A80100206B65792025732063726561747F
:1089000065642E2E2E2C2076616C756520257320D3
:108910000A0000002DE9F041AEB004460120FAF74C
:108920003FFF9620FCF796F848A0FAF747FF9620FD
:10893000FCF790F80020FAF733FF0CB149480460C7
:108940000025002648A0FFF76BFF05464AA0FFF769
:1089500067FF064605B1B6B90120FAF721FF962058
:10896000FCF778F849A0FAF729FF9620FCF772F88F
:108970000020FAF715FF6FF001003A4909688847AF
:108980002EB0BDE8F0812846F7F771FC07464C4948
:1089900003C9CDE92C012D974949083103C9CDE917
:1089A0002A012B964649103103C9CDE92801182226
:1089B0004349183122A8F7F7C5FB2CA823902AA910
:1089C00022A8C16028A941613D49303103C9CDE9E0
:1089D000200122A821904FF48070FDF75DFD3949F8
:1089E00008604FF480720846016820A800F002FA7F
:1089F00080460120FAF7D4FE9620FCF72BF8314888
:108A0000016831A0FAF7DAFE9620FCF723F800207F
:108A1000FAF7C6FE80216846F7F7AFFB33A23BA109
:108A20006846FAF7DBFE414A264801686846FFF7C8
:108A3000A2FC2448006830B122480068FCF752F9D3
:108A400000202049086000BF9AE70000626567695E
:108A50006E206C6F67696E206465766963652E2E83
:108A60002E0A00007001002070616E646F5F646503
:108A7000766963655F69640070616E646F5F6465E9
:108A8000766963655F736563726574006C6F6769AF
:108A90006E206661696C6564202120646576696377
:108AA0006520686173206E6F74206265656E207248
:108AB00065676973746572642E2E2E0A00000000CB
:108AC000C4A0000874010020646576696365206CA9
:108AD0006F67696E20726571756573743A3A3A0A08
:108AE00025730A28656E64290A0000006874747092
:108AF0003A2F2F3232322E3137352E3132392E3154
:108B000039343A31383038380000000025732F7678
:108B1000312F646576696365732F61757468656E5E
:108B20007469636174696F6E000000002D52000863
:108B30002DE9F041BAB004460120FAF731FE962043
:108B4000FBF788FF4EA0FAF739FE9620FBF782FF6D
:108B50000020FAF725FE0CB15148046000250026DC
:108B6000002750A0FFF75CFE054652A0FFF758FE15
:108B7000064655A0FFF754FE074636A8FCF720F935
:108B800000208DF8E7000120FAF70AFE9620FBF797
:108B900061FF36A951A0FAF711FE9620FBF75AFFA4
:108BA0000020FAF7FDFD524903C9CDE934015049CF
:108BB000083103C9CDE9320136A833904C49103150
:108BC00003C9CDE930014A49183103C9CDE92E0165
:108BD0004749203103C9CDE92C01282244492831D5
:108BE00022A8F7F7AFFA34A8239032A922A8C160CF
:108BF00030A941612EA9C1612CA941623C49503183
:108C000003C9CDE9200122A821904FF48070FDF71F
:108C100043FC384908604FF480720846016820A878
:108C200000F0E8F880460120FAF7BAFD9620FBF73D
:108C300011FF3048016830A0FAF7C0FD9620FBF71D
:108C400009FF0020FAF7ACFD80216846F7F795FA96
:108C500033A23BA16846FAF7C1FD404A25480168A6
:108C60006846FFF788FB2348006830B12148006858
:108C7000FCF738F800201F4908603AB0BDE8F081E1
:108C800050414E444F20626567696E207265676986
:108C900073746572206465766963652E2E2E0A00F2
:108CA0007801002070616E646F5F6465766963654A
:108CB0005F69640070616E646F5F646576696365A7
:108CC0005F7365637265740070616E646F5F646585
:108CD000766963655F6B657900000000646576699D
:108CE00063655F73657269616C3A25730A00000001
:108CF000FCA000087C010020646576696365207231
:108D00006567697374657220726571756573743A0D
:108D10003A3A0A25730A28656E64290A00000000A1
:108D2000687474703A2F2F3232322E3137352E312B
:108D300032392E3139343A313830383800000000B9
:108D400025732F76312F646576696365732F72659D
:108D500067697374726174696F6E0000B9540008BA
:108D600010B500F007F802490120FFF7F7FB10BD2E
:108D70003D93000810B50120FAF712FD9620FBF78D
:108D800069FE12A0FAF71AFD9620FBF763FE002099
:108D9000FAF706FD002014490870FDF78BFA00F081
:108DA0009BFB41F2883011490880012088701048EF
:108DB00048600220C870084600F030FB0B4800F005
:108DC0006FFB0A4800F050FB10BD000050414E44BC
:108DD0004F206761746577617920696E6974696194
:108DE0006C2E2E2E2E0A000080010020F410002090
:108DF0004D4B000870B592B005460C4616461CB99E
:108E00004FF0FF3012B070BD0D4804600D48066091
:108E100000200D49086000956846FDF705FA0B48EB
:108E20000F9000BF6846FDF751F90028FAD10449B8
:108E30000968054A1268885403480068E2E70000A0
:108E400084010020880100208C010020A95E000818
:108E500001460878074A1268904201D10020704705
:108E60000A78501C087002EB4200034A02EB8000B3
:108E7000F5E70000A4010020C01100202DE9FE4309
:108E800004460E466068618845186068218800EBDA
:108E900001082F463846FBF761FB18B14FF0FF3051
:108EA000BDE8FE831935454511D90120FAF778FC54
:108EB0009620FBF7CFFD10A0FAF780FC9620FBF779
:108EC000C9FD0020FAF76CFC4FF0FF30E8E720887E
:108ED0006188401A83B2324639466846FCF748FE3C
:108EE0000C3D00982860019868600298A86060882E
:108EF0000D3060800020D3E7496E636F7272656346
:108F000074206465636F64652062756666657220AF
:108F10006C656E6774682E0A000000002DE9F04150
:108F20008AB004460D4660686188461860682188EA
:108F300000EB0108374606F10C000646404513D900
:108F40000120FAF72DFC9620FBF784FD1FA0FAF70D
:108F500035FC9620FBF77EFD0020FAF721FC4FF050
:108F6000FF300AB0BDE8F081788828802888FFF7B4
:108F700021F92880F888ADF80600BDF80600FFF753
:108F800019F9ADF80600694603A8FCF759FE88B147
:108F90000120FAF705FC9620FBF75CFD14A0FAF718
:108FA0000DFC9620FBF756FD0020FAF7F9FB4FF079
:108FB000FF30D6E7193E192203A93046F7F7C2F869
:108FC00060880D3860800020CBE70000496E636F39
:108FD000727265637420656E636F64652062756686
:108FE000666572206C656E6774682E0A000000006A
:108FF000496E697420706462696E20686561646599
:1090000072206661696C65642E0A000070B50546C1
:109010000C4668681930698846188EB90120FAF73D
:10902000BFFB9620FBF716FD09A0FAF7C7FB9620B9
:10903000FBF710FD0020FAF7B3FB4FF0FF3070BDD7
:10904000308820802088FFF7B5F820800020F6E7E0
:10905000737562646576696365206E756C6C0A0071
:109060000FB410B5342202A90C48F7F76BF898B981
:109070000120FAF795FB9620FBF7ECFC08A0FAF725
:109080009DFB9620FBF7E6FC0020FAF789FB4FF0EA
:10909000FF3010BC5DF814FB0020FAE7001100203F
:1090A00070616E646F5F70726F746F636F6C5F6915
:1090B0006E6974206661696C65642E0A00000000A8
:1090C00073B5044660681930618845188DB9012070
:1090D000FAF766FB9620FBF7BDFC13A0FAF76EFBD0
:1090E0009620FBF7B7FC0020FAF75AFB4FF0FF3051
:1090F0007CBD0120FAF754FB9620FBF7ABFCBDF8D2
:1091000004100DA0FAF75AFB9620FBF7A3FC0020F1
:10911000FAF746FBBDF80400FFF74CF80190BDF8E4
:10912000040028800020E3E7737562646576696354
:1091300065206E756C6C0A00736574207375625FD0
:109140006465766963655F69642025640A000000D0
:109150002DE9FF4106460D460120FAF721FB962036
:10916000FBF778FC4CA0FAF729FB9620FBF772FC82
:109170000020FAF715FB002400270020039005F1DA
:109180000D0087B20D213846FFF7F2F904466068FA
:1091900088B90120FAF704FB9620FBF75BFC4549F0
:1091A00045A0FAF70BFB9620FBF754FC0020FAF7DA
:1091B000F7FABDE8FF816168628888182A4631465F
:1091C000F6F7C0FF03A92046FFF7A8FE78B10120FB
:1091D000FAF7E6FA9620FBF73DFC3CA0FAF7EEFA28
:1091E0009620FBF737FC0020FAF7DAFAE1E70121D5
:1091F0002046FFF765FF2188606800F0C7FABDF8D8
:109200000C00012804D0022806D003280CD107E066
:1092100036A0006802901AE035A00068029016E0BF
:1092200034A00068029012E00120FAF7B9FA962003
:10923000FBF710FC30A0FAF7C1FA9620FBF70AFC06
:109240000020FAF7ADFA2046FFF7AFF9B1E700BF0B
:109250002E4890F8B0000F280AD100200121CDE956
:1092600000102388626802A92848F9F7B1F90EE0D6
:109270000120FAF795FA9620FBF7ECFB24A0FAF709
:109280009DFA9620FBF7E6FB0020FAF789FA2046C4
:10929000FFF78BF900BF8CE770616E646F5F7075CC
:1092A000626C6973685F646174615F6368616E6E4C
:1092B000656C3100A8A0000825733A6D616C6C6F75
:1092C00063206661696C65642E0A000070616E64DB
:1092D0006F5F70726F746F636F6C5F656E636F64E6
:1092E00065206572726F722E0A0000006300000034
:1092F00065000000730000006572726F722070617B
:10930000796C6F616420747970650A001010002018
:109310004D515454207374617465206973206E6FCD
:1093200074206176616961626C6520666F7220707D
:1093300075626C6973682F6E000000002DE9F041C2
:1093400007460D460FB9BDE8F0810120FAF728FA6B
:109350009620FBF77FFB22A0FAF730FA9620FBF766
:1093600079FB0020FAF71CFA2946384600F00EFA7D
:109370000620FDF791F8044625802846FDF78CF875
:10938000C4F80200D4F802002A463946F6F7DAFE9D
:109390002046FBF76FFD0646012E05D0032E07D1B0
:1093A0002046FBF701FB14E02046FBF78BFA10E0A8
:1093B0000120FAF7F5F99620FBF74CFB314610A097
:1093C000FAF7FCF99620FBF745FB0020FAF7E8F9DD
:1093D00000BF00BF2046FBF761FB00BFB3E7000002
:1093E0007375626465766976652072656365697612
:1093F000652061207061636B6167653A200A000037
:10940000756E7375706F727465642070616C6F61D6
:10941000642074797065203A2025640010B50446F4
:10942000E078012805D109480460204600F0C8FB17
:109430000AE0E078022804D10548046000F052FCFC
:1094400002E004A0FAF7BAF910BD0000AC01002058
:10945000B001002077726F6E672074696D657220AD
:109460006E6F210A0000000010B50446E078012864
:1094700002D100F0D9FB08E0E078022802D100F028
:1094800069FC02E001A0FAF799F910BD77726F6EDE
:10949000672074696D6572206E6F210A00000000FC
:1094A00010B50446E078012802D100F0C5FB08E0C1
:1094B000E078022802D100F055FC02E001A0FAF7A2
:1094C0007DF910BD77726F6E672074696D657220CB
:1094D0006E6F210A0000000010B502490020FFF75E
:1094E0003DF810BDA19E00080020014670470146CE
:1094F000C86808B900207047C868401EC86001F1FC
:109500001A00CA68805CF6E770B50E4804680CB9AA
:10951000002070BDA66846B925680020094908608A
:109520002046FBF7DFFB2846F3E725680548066081
:109530000020044909684860A0602046FBF7D2FB80
:109540002846E6E720000020024602F11A00D36810
:10955000C154D068401CD06000201076D0680A2822
:1095600001DA012070470020FCE70000014A116089
:109570007047000038000020014A11607047000069
:1095800044000020014A11607047000040000020A4
:10959000014A1160704700003C00002038B50120EE
:1095A000FAF7FEF89620FBF755FA1BA0FAF706F932
:1095B0009620FBF74FFA0020FAF7F2F8002000900F
:1095C0001C48046811E09DF8001001EB41110C22C9
:1095D00002EB810188B284222146F6F7C5FF9DF88F
:1095E0000000401CC0B200902468002CEBD1012286
:1095F00069460B20F6F7B8FF0120FAF7D1F896205C
:10960000FBF728FA0CA0FAF7D9F89620FBF722FA14
:109610000020FAF7C5F838BD736176696E6720647B
:1096200061746120746F20666C6173682E2E2E0A3F
:1096300000000000A8010020646F6E652E2E2E0A27
:109640000000000070B504462046F6F7C9FD85B25B
:1096500029462046FAF782F870BD00002DE9F04156
:109660000020FBF71BF8044684B90120FAF798F8AC
:109670009620FBF7EFF92CA0FAF7A0F89620FBF75D
:10968000E9F90020FAF78CF8BDE8F0810025FBF736
:1096900059F8804630E0FBF75FF806467EB90120B6
:1096A000FAF77EF89620FBF7D5F926A0FAF786F8A8
:1096B0009620FBF7CFF90020FAF772F8E4E730467E
:1096C00069688847297832462046FAF7E5FA07465E
:1096D00077B10120FAF764F89620FBF7BBF921A0D7
:1096E000FAF76CF89620FBF7B5F90020FAF758F86E
:1096F0003046FBF7ECF900BF4046FFF7A9FB051E1B
:10970000C9D14046FBF7DCF92288D4F802100120C9
:10971000FAF7CEFE2188D4F8020000F037F8204690
:10972000FBF7BCF900BFAFE7637265617465206445
:10973000617461207061636B616765206572726F2F
:10974000720A000043726561746520706172616D18
:109750007320626C6F636B206661696C65642E0AAE
:10976000000000006164645F6E6578745F70726F02
:109770007065727479206661696C65642E00000002
:1097800001490870704700005001002070B505467F
:109790000E4600240120FAF703F89620FBF75AF949
:1097A000314617A0FAF70AF89620FBF753F9002084
:1097B000F9F7F6FF00BF10E00120F9F7F1FF96205E
:1097C000FBF748F9295D17A0F9F7F8FF9620FBF79A
:1097D00041F90020F9F7E4FF641CB442ECDB0120FE
:1097E000F9F7DEFF9620FBF735F910A0F9F7E6FF51
:1097F0009620FBF72FF90020F9F7D2FF70BD00008B
:109800005061636B616765206C656E6774683A20B0
:1098100025640A636F6E74656E742069733A200A5A
:109820000000000025303278200000000A0000000F
:1098300070B505460E4600240120F9F7B1FF9620C9
:10984000FBF708F9314617A0F9F7B8FF9620FBF7A8
:1098500001F90020F9F7A4FF00BF10E00120F9F79B
:109860009FFF9620FBF7F6F8295D17A0F9F7A6FFF2
:109870009620FBF7EFF80020F9F792FF641CB44242
:10988000ECDB0120F9F78CFF9620FBF7E3F810A042
:10989000F9F794FF9620FBF7DDF80020F9F780FF39
:1098A00070BD00005061636B616765206C656E6719
:1098B00074683A2025640A636F6E74656E7420695B
:1098C000733A200A000000002530327820000000A2
:1098D0000A00000002E04268521C4260D0E9012305
:1098E0009A4206DAD0E90023D15C2029F3D00A2974
:1098F000F1D070472DE9FE4381460E46274A07CA3C
:109900008DE807004FF0FF370025344600E0641C67
:1099100020780D28FBD020780A28F8D0002509E00F
:109920005DF825102046F6F733FC08B16FB203E06E
:10993000681CC5B2032DF3D300BF27B1012F1BD084
:10994000022F24D122E016A12046F6F721FC04467E
:109950000C342046F6F77EFC8046B8F1000F07D1A4
:109960001348006820B100210846114A1268904748
:109970000120104908700BE04FF0FF3100200C4A25
:109980001268904701200B49087001E000E000BF19
:1099900000BF0848007840B2BDE8FE833CA0000844
:1099A0002B4349504F50454E3A20312C00000000C7
:1099B000380000205101002070B504460D460E49C4
:1099C0000EA0F9F7FBFE2E46601C18B913A0F9F79C
:1099D000F5FE10E0174850F8240060B1154850F823
:1099E0002400406938B1134951F8240051F824107B
:1099F0004A693146904770BD82A1000825732C64E6
:109A0000656275673A6E657420636F6E6E65637428
:109A10002063616C6C6261636B0A00006D6F64753A
:109A20006C652063616C6C6261636B206572726F40
:109A300072210A008012002070B504460D460648C7
:109A4000006828B14FF0FF310020034A12689047A8
:109A50004FF0FF3070BD00004400002070B5044698
:109A60000D460E490EA0F9F7A9FE601C18B913A007
:109A7000F9F7A4FE10E01A4850F8240060B1184825
:109A800050F82400006A38B1154951F8240051F803
:109A900024100A6A2946904770BD0000ABA1000857
:109AA00025732C64656275673A6E6574206469730A
:109AB000636F6E656374206F6B0A00006D6F647571
:109AC0006C6520646973636F6E6E65637420636197
:109AD0006C6C6261636B206572726F72210A0000A8
:109AE000801200207CB504460D4616460195ADF85F
:109AF0000060601C18B90BA0F9F760FE10E0114877
:109B000050F8240060B10F4850F82400806938B143
:109B10000C4951F8240051F824108A69694690478D
:109B20007CBD00006D6F64756C6520726563762086
:109B300063616C6C6261636B206572726F72210A83
:109B4000000000008012002070B504460D460E494A
:109B50000EA0F9F733FE2E46601C18B911A0F9F7D4
:109B60002DFE10E0154850F8240060B1134850F85D
:109B70002400C06938B1114951F8240051F824106B
:109B8000CA693146904770BD99A1000825732C64BD
:109B9000656275673A6E65745F746370206F6B0AF7
:109BA000000000006D6F64756C652063616C6C6211
:109BB00061636B206572726F72210A00801200204F
:109BC00038B5044600BF1648C06940F00200144989
:109BD000C8610846C06900F00200009000BF00BFE5
:109BE000062205211C20F7F7B6F91C20F7F7A6F985
:109BF0004FF080400B49086048F69F4048600021C4
:109C00000848816020884000401E0649C860002145
:109C100004480161F7F787FD00F00EF838BD000039
:109C200000100240A812002010B50248F7F7ACFD62
:109C300010BD0000A812002010B50248F7F7B3FDD0
:109C400010BD0000A8120020F8B504460D461646C7
:109C5000174805701748066000BF1748C06940F0F4
:109C600002001549C8610846C06900F00200009072
:109C700000BF00BF032211461D20F7F76CF91D201D
:109C8000F7F75CF90D480E49086048F69F404860B8
:109C900000210B4881606000401E0949C860002116
:109CA00007480161F7F73FFD00F014F8F8BD000028
:109CB0002400002028000020001002400004004082
:109CC0008405002010B50248F7F75EFD10BD0000C6
:109CD0008405002010B50248F7F765FD10BD0000AF
:109CE0008405002008B500BF1648C06940F0040094
:109CF0001449C8610846C06900F00400009000BF24
:109D000000BF062205211E20F7F725F91E20F7F7D0
:109D100015F90D480D49086048F69F40486000213C
:109D20000A4881600A48006800884000401E0749D0
:109D3000C860002105480161F7F7F5FC00F012F852
:109D400008BD00000010024000080040E81200209A
:109D5000B001002010B50248F7F716FD10BD000055
:109D6000E812002010B50248F7F71DFD10BD0000F5
:109D7000E812002010B50446F8F730FE11481249E9
:109D800008600846446000218160C16001610C21C7
:109D9000416100218161F7F707FE18B163210BA033
:109DA000F9F70AFD08480068C06840F0100006494D
:109DB0000968C8604FF4FA720A490348F7F730FFA0
:109DC00010BD0000004400407C0400202E2E5C5397
:109DD000595354454D5C55736172745C757361726F
:109DE000742E6300C001002010B5044609480A49DA
:109DF00008600846446000218160C16001618161A2
:109E00000C214161F7F7D0FD012204490248F7F720
:109E100069FF10BD00480040BC040020180000206D
:109E200070B505460C460120F9F7BAFC9620FAF702
:109E300011FE214605A0F9F7C1FC9620FAF70AFEAB
:109E40000020F9F7ADFC002070BD000075726320A2
:109E500068616E646C65723A2025730A0000000028
:109E600038B5054600240020009000BF11E00B4AE1
:109E700052F834102868F6F7BAF940B9074800EBF1
:109E8000C4002968426868469047002038BD601CBD
:109E9000C4B2082CEBD34FF0FF30F7E710010020DD
:109EA0002DE9FF4706460D460027B8460620FCF779
:109EB000F3FA04468CB90120F9F772FC9620FAF700
:109EC000C9FD324932A0F9F779FC9620FAF7C2FDB4
:109ED0000020F9F765FCBDE8FF872846FCF7DCFAAF
:109EE000C4F80200D4F8020098B90120F9F758FC30
:109EF0009620FAF7AFFD254925A0F9F75FFC9620DB
:109F0000FAF7A8FD0020F9F74BFC2046FAF7EAFE25
:109F1000E1E7D4F802002A463146F6F713F9258026
:109F200002A92046FAF780FF8146BDF80A004FF6E5
:109F3000FB71884218D10120F9F732FC9620FAF71C
:109F400089FD18A0F9F73AFC9620FAF783FD002066
:109F5000F9F726FC4846FAF75AFFCDE90001082137
:109F60006846FFF713FC00BFD4F8020030B1D4F804
:109F70000200FAF7B7FE0020C4F802001CB1204628
:109F8000FAF7B0FE002400BFA5E7000054A10008C6
:109F900025733A6D616C6C6F63206572726F72210C
:109FA0000A00000050414E444F3A2073796E6368B6
:109FB000726F6E697A652074696D650A0000000031
:109FC0000003030601040602050003051F1C1F1EF3
:109FD0001F1E1F1F1E1F1E1FC8A3000838A4000835
:109FE000ECA20008C8A3000838A4000890A200084A
:109FF000C8A3000838A4000898A20008C8A3000855
:10A0000038A40008A0A20008ACA20008C8A3000859
:10A0100038A400089CA30008C8A3000838A40008BE
:10A02000C8A3000838A4000884A20008C8A3000838
:10A0300038A4000878A20008ACA20008B8A2000862
:10A0400038A40008C8A300086CA2000838A40008BF
:10A0500028A30008C8A300081CA30008D8A3000870
:10A06000C8A3000838A4000878A4000828A30008A2
:10A07000C8A3000838A40008FCA2000858A20008E1
:10A0800064A40008C8A2000838A40008DCA20008E4
:10A090000000000000000000010203040607080998
:10A0A000000000000102030470616E646F5F707550
:10A0B000626C6973685F646174615F6368616E6E2E
:10A0C000656C310049000000000000002200000023
:10A0D00000000000220000001CA50008F4A40008F5
:10A0E000000000000CA500080000000000A500080A
:10A0F000000000007B0300000000000022000000C0
:10A100005CA50008220000000000000049000000DB
:10A11000010000002200000024A500082200000029
:10A120002CA50008A8A500080000000034A5000820
:10A130000000000050A500080000000040A5000835
:10A1400000000000A0A50008000000007B05000042
:10A15000000000007A65726F5F6465766963655F11
:10A16000646174615F70726F63657373006D7174A5
:10A17000745F74696D6572004D5154545F5461731E
:10A180006B007463705F636F6E6E65637465645FAC
:10A1900063616C6C6261636B007463705F73656EA6
:10A1A000745F63616C6C6261636B007463705F64A5
:10A1B0006973636F6E6E65637465645F63616C6C15
:10A1C0006261636B006E65745F7463705F73656E6C
:10A1D00064000040404040404040404041414141D7
:10A1E000414040404040404040404040404040406E
:10A1F0004040400502020202020202020202020282
:10A200000202022020202020202020202002020202
:10A210000202020290909090909010101010101076
:10A22000101010101010101010101010101002024A
:10A2300002020202888888888888080808080808B6
:10A24000080808080808080808080808080802029A
:10A2500002024000D3A100082B4343485F5045450C
:10A26000525F434C4F5345443A2000002B43495022
:10A2700053454E443A2000002B4E4554434C4F5317
:10A28000453A20002B4E45544F50454E3A20000091
:10A290002B4350494E3A20002B4353513A200000A3
:10A2A0002B4950414444523A200000002B49502091
:10A2B0004552524F523A20002B4349504F50454E81
:10A2C0003A20312C000000002B43485454504143A5
:10A2D000543A20444154412C000000002B43485480
:10A2E00054504143543A2030000000002B4343486F
:10A2F00053544152543A2030000000002B4343484D
:10A3000053454E443A0000002B4950434C4F5345AF
:10A310003A0000002B5354494E3A00002B43495059
:10A320004552524F523A00003E00000041542B4328
:10A330005053493F0000000041542B494643000060
:10A3400041542B43434853454E44000041542B4352
:10A35000495053454E44000041542B4349504D4F02
:10A3600044450000504220444F4E4500534D532079
:10A37000444F4E450000000041542B434348434C9A
:10A380004F53450041542B434950434C4F534500D4
:10A3900041542B4E4554434C4F53450041544500C6
:10A3A00041542B43524547004F504C205550444197
:10A3B00054494E4700000000504E4E205550444135
:10A3C00054494E47000000004F4B000041542B43BE
:10A3D00043484F50454E00002B4343484F50454E95
:10A3E0000000000041542B4349504F50454E00009F
:10A3F00041542B4E45544F50454E000041542B4381
:10A4000050494E0041542B4347534E0041542B4377
:10A41000495053524950000041542B434348535430
:10A420004F50000041542B435351000041542B49DD
:10A4300050414444520000004552524F5200000027
:10A4400041542B43485454504143540041542B43EE
:10A45000434853455400000041542B434348535450
:10A46000415254002B43485454504143543A2052D3
:10A4700045515545535400002B43434852454356DC
:10A48000000000002B4350494E3A205245414459A8
:10A490000000000052445900504F535420257320AF
:10A4A000485454502F312E310D0A486F73743A209E
:10A4B00025733A25640D0A4163636570743A2A2F47
:10A4C0002A0D0A436F6E6E656374696F6E3A20637E
:10A4D0006C6F73650D0A557365722D4167656E74F7
:10A4E0003A2053494D373630300D0A25730D0A2571
:10A4F000730000006465766963655F69640000004D
:10A5000070726F746F636F6C000000006465766931
:10A5100063655F7365637265740000006D717474C8
:10A520000000000053494D3736303000302E302EB9
:10A53000310000006465766963655F636F64650080
:10A540006465766963655F6D6F64756C65000000B6
:10A550006465766963655F74797065003435343895
:10A560006363653935656533303937623433346157
:10A57000313435353434356531303862363762340C
:10A5800030633065333835313062393932323562D3
:10A59000306464636561363035343866000000002D
:10A5A00076657273696F6E0070726F647563745F45
:10A5B0006B657900636C69656E742D3E636F6E6EBA
:10A5C00073746174653A25642C20747970653A253A
:10A5D000642C20516F733A25642C2069643A2564F9
:10A5E0002C206D657373616765206C656E67746898
:10A5F0003A25640A0000000018A6000800000020A8
:10A60000C001000062040008C8A60008C0010020C4
:10A61000683500001C380008413210024701139CC5
:10A62000A3140811401B08380813913F2B08FC1095
:10A6300012461C0824A41012471B080408132551B5
:10A640005B0858201AF008138D831B08900813D15B
:10A65000825B08A0186A2C081930136D501B084043
:10A66000081345581B08E41813F5981B084C0813E9
:10A67000A15C5B0884282A0C6019086910295029FC
:10A68000085A4C185A58081ACC181B51415019082E
:10A690001ACD085A78285A18201A08101B399A48D7
:10A6A000191013219E1B08141029085A94105AA837
:10A6B000105AB8085A6C085A6408F3FF01042CA217
:08A6C0004A041AFF01012C00FD
:04000005080000ED02
:00000001FF
